Archive member included because of file (symbol)

C:/Program Files/Microchip/MPLAB C32/bin/../lib/gcc/pic32mx/3.4.4/size\libgcc.a(_udivdi3.o)
                              ..\Microchip\TCPIP Stack\Objects - TCPIP Demo App-C32\Tick.o (__udivdi3)
C:/Program Files/Microchip/MPLAB C32/bin/../lib/gcc/pic32mx/3.4.4/../../../../pic32mx/lib/size\libc.a(memcmp.o)
                              Objects - TCPIP Demo App-C32\CustomHTTPApp.o (memcmp)
C:/Program Files/Microchip/MPLAB C32/bin/../lib/gcc/pic32mx/3.4.4/../../../../pic32mx/lib/size\libc.a(memcpy.o)
                              Objects - TCPIP Demo App-C32\MainDemo.o (memcpy)
C:/Program Files/Microchip/MPLAB C32/bin/../lib/gcc/pic32mx/3.4.4/../../../../pic32mx/lib/size\libc.a(memset.o)
                              ..\Microchip\TCPIP Stack\Objects - TCPIP Demo App-C32\DHCP.o (memset)
C:/Program Files/Microchip/MPLAB C32/bin/../lib/gcc/pic32mx/3.4.4/../../../../pic32mx/lib/size\libc.a(strcmp.o)
                              Objects - TCPIP Demo App-C32\CustomHTTPApp.o (strcmp)
C:/Program Files/Microchip/MPLAB C32/bin/../lib/gcc/pic32mx/3.4.4/../../../../pic32mx/lib/size\libc.a(strcpy.o)
                              Objects - TCPIP Demo App-C32\MainDemo.o (strcpy)
C:/Program Files/Microchip/MPLAB C32/bin/../lib/gcc/pic32mx/3.4.4/../../../../pic32mx/lib/size\libc.a(strlen.o)
                              Objects - TCPIP Demo App-C32\MainDemo.o (strlen)
C:/Program Files/Microchip/MPLAB C32/bin/../lib/gcc/pic32mx/3.4.4/../../../../pic32mx/lib/size\libc.a(general-exception.o)
                              C:/Program Files/Microchip/MPLAB C32/bin/../lib/gcc/pic32mx/3.4.4/../../../../pic32mx/lib/size/crt0.o (_general_exception_context)
C:/Program Files/Microchip/MPLAB C32/bin/../lib/gcc/pic32mx/3.4.4/../../../../pic32mx/lib/size\libc.a(strchr.o)
                              ..\Microchip\TCPIP Stack\Objects - TCPIP Demo App-C32\SMTP.o (strchr)
C:/Program Files/Microchip/MPLAB C32/bin/../lib/gcc/pic32mx/3.4.4/../../../../pic32mx/lib/size\libc.a(strstr.o)
                              ..\Microchip\TCPIP Stack\Objects - TCPIP Demo App-C32\SMTP.o (strstr)
C:/Program Files/Microchip/MPLAB C32/bin/../lib/gcc/pic32mx/3.4.4/../../../../pic32mx/lib/size\libc.a(exit.o)
                              C:/Program Files/Microchip/MPLAB C32/bin/../lib/gcc/pic32mx/3.4.4/../../../../pic32mx/lib/size/crt0.o (exit)
C:/Program Files/Microchip/MPLAB C32/bin/../lib/gcc/pic32mx/3.4.4/../../../../pic32mx/lib/size\libc.a(rand.o)
                              ..\Microchip\TCPIP Stack\Objects - TCPIP Demo App-C32\Helpers.o (rand)
C:/Program Files/Microchip/MPLAB C32/bin/../lib/gcc/pic32mx/3.4.4/../../../../pic32mx/lib/size\libc.a(atol.o)
                              ..\Microchip\TCPIP Stack\Objects - TCPIP Demo App-C32\HTTP2.o (atol)
C:/Program Files/Microchip/MPLAB C32/bin/../lib/gcc/pic32mx/3.4.4/../../../../pic32mx/lib/size\libc.a(atoi.o)
                              ..\Microchip\TCPIP Stack\Objects - TCPIP Demo App-C32\SMTP.o (atoi)
C:/Program Files/Microchip/MPLAB C32/bin/../lib/gcc/pic32mx/3.4.4/../../../../pic32mx/lib/size\libc.a(strtol.o)
                              C:/Program Files/Microchip/MPLAB C32/bin/../lib/gcc/pic32mx/3.4.4/../../../../pic32mx/lib/size\libc.a(atol.o) (strtol)
C:/Program Files/Microchip/MPLAB C32/bin/../lib/gcc/pic32mx/3.4.4/../../../../pic32mx/lib/size\libc.a(_iobdata.o)
                              C:/Program Files/Microchip/MPLAB C32/bin/../lib/gcc/pic32mx/3.4.4/../../../../pic32mx/lib/size\libc.a(exit.o) (_libc_data)
C:/Program Files/Microchip/MPLAB C32/bin/../lib/gcc/pic32mx/3.4.4/../../../../pic32mx/lib/size\libc.a(_iobfuncs.o)
                              C:/Program Files/Microchip/MPLAB C32/bin/../lib/gcc/pic32mx/3.4.4/../../../../pic32mx/lib/size\libc.a(_iobdata.o) (_filbuf_simple)
C:/Program Files/Microchip/MPLAB C32/bin/../lib/gcc/pic32mx/3.4.4/../../../../pic32mx/lib/size\libc.a(stubs.o)
                              C:/Program Files/Microchip/MPLAB C32/bin/../lib/gcc/pic32mx/3.4.4/../../../../pic32mx/lib/size\libc.a(exit.o) (pthread_mutex_lock)
C:/Program Files/Microchip/MPLAB C32/bin/../lib/gcc/pic32mx/3.4.4/../../../../pic32mx/lib/size\libc.a(default-bootstrap-exception-handler.o)
                              C:/Program Files/Microchip/MPLAB C32/bin/../lib/gcc/pic32mx/3.4.4/../../../../pic32mx/lib/size/crt0.o (_bootstrap_exception_handler)
C:/Program Files/Microchip/MPLAB C32/bin/../lib/gcc/pic32mx/3.4.4/../../../../pic32mx/lib/size\libc.a(default-on-reset.o)
                              C:/Program Files/Microchip/MPLAB C32/bin/../lib/gcc/pic32mx/3.4.4/../../../../pic32mx/lib/size/crt0.o (_on_reset)
C:/Program Files/Microchip/MPLAB C32/bin/../lib/gcc/pic32mx/3.4.4/../../../../pic32mx/lib/size\libc.a(default-on-bootstrap.o)
                              C:/Program Files/Microchip/MPLAB C32/bin/../lib/gcc/pic32mx/3.4.4/../../../../pic32mx/lib/size/crt0.o (_on_bootstrap)
C:/Program Files/Microchip/MPLAB C32/bin/../lib/gcc/pic32mx/3.4.4/../../../../pic32mx/lib/size\libc.a(default-nmi-handler.o)
                              C:/Program Files/Microchip/MPLAB C32/bin/../lib/gcc/pic32mx/3.4.4/../../../../pic32mx/lib/size/crt0.o (_nmi_handler)
C:/Program Files/Microchip/MPLAB C32/bin/../lib/gcc/pic32mx/3.4.4/../../../../pic32mx/lib/size\libc.a(_mon_getc.o)
                              C:/Program Files/Microchip/MPLAB C32/bin/../lib/gcc/pic32mx/3.4.4/../../../../pic32mx/lib/size\libc.a(_iobfuncs.o) (_mon_getc)
C:/Program Files/Microchip/MPLAB C32/bin/../lib/gcc/pic32mx/3.4.4/../../../../pic32mx/lib/size\libc.a(_mon_write.o)
                              C:/Program Files/Microchip/MPLAB C32/bin/../lib/gcc/pic32mx/3.4.4/../../../../pic32mx/lib/size\libc.a(_iobfuncs.o) (_mon_write)
C:/Program Files/Microchip/MPLAB C32/bin/../lib/gcc/pic32mx/3.4.4/../../../../pic32mx/lib/size\libc.a(_exit.o)
                              C:/Program Files/Microchip/MPLAB C32/bin/../lib/gcc/pic32mx/3.4.4/../../../../pic32mx/lib/size\libc.a(exit.o) (_exit)
C:/Program Files/Microchip/MPLAB C32/bin/../lib/gcc/pic32mx/3.4.4/../../../../pic32mx/lib/size\libc.a(ctype.o)
                              C:/Program Files/Microchip/MPLAB C32/bin/../lib/gcc/pic32mx/3.4.4/../../../../pic32mx/lib/size\libc.a(strtol.o) (_ctype)
C:/Program Files/Microchip/MPLAB C32/bin/../lib/gcc/pic32mx/3.4.4/../../../../pic32mx/lib/size\libc.a(errno.o)
                              C:/Program Files/Microchip/MPLAB C32/bin/../lib/gcc/pic32mx/3.4.4/../../../../pic32mx/lib/size\libc.a(strtol.o) (errno)
C:/Program Files/Microchip/MPLAB C32/bin/../lib/gcc/pic32mx/3.4.4/../../../../pic32mx/lib/size\libc.a(_mon_putc.o)
                              C:/Program Files/Microchip/MPLAB C32/bin/../lib/gcc/pic32mx/3.4.4/../../../../pic32mx/lib/size\libc.a(_mon_write.o) (_mon_putc)
C:/Program Files/Microchip/MPLAB C32/bin/../lib/gcc/pic32mx/3.4.4/../../../../pic32mx/lib/size\libmchp_peripheral.a(int_disable_interrupts_lib.o)
                              Objects - TCPIP Demo App-C32\MainDemo.o (INTDisableInterrupts)
C:/Program Files/Microchip/MPLAB C32/bin/../lib/gcc/pic32mx/3.4.4/../../../../pic32mx/lib/size\libmchp_peripheral.a(int_enable_mv_int_lib.o)
                              Objects - TCPIP Demo App-C32\MainDemo.o (INTEnableSystemMultiVectoredInt)
C:/Program Files/Microchip/MPLAB C32/bin/../lib/gcc/pic32mx/3.4.4/../../../../pic32mx/lib/size\libmchp_peripheral.a(int_restore_interrupts_lib.o)
                              Objects - TCPIP Demo App-C32\MainDemo.o (INTRestoreInterrupts)
C:/Program Files/Microchip/MPLAB C32/bin/../lib/gcc/pic32mx/3.4.4/../../../../pic32mx/lib/size\libmchp_peripheral.a(soft_reset_lib.o)
                              ..\Microchip\TCPIP Stack\Objects - TCPIP Demo App-C32\ENC28J60.o (SoftReset)
C:/Program Files/Microchip/MPLAB C32/bin/../lib/gcc/pic32mx/3.4.4/../../../../pic32mx/lib/size\libmchp_peripheral.a(pcache.o)
                              Objects - TCPIP Demo App-C32\MainDemo.o (CheKseg0CacheOn)
C:/Program Files/Microchip/MPLAB C32/bin/../lib/gcc/pic32mx/3.4.4/../../../../pic32mx/lib/size\libmchp_peripheral.a(int_enable_interrupts_lib.o)
                              C:/Program Files/Microchip/MPLAB C32/bin/../lib/gcc/pic32mx/3.4.4/../../../../pic32mx/lib/size\libmchp_peripheral.a(int_enable_mv_int_lib.o) (INTEnableInterrupts)

Allocating common symbols
Common symbol       size              file

UDPTxCount          0x2               ..\Microchip\TCPIP Stack\Objects - TCPIP Demo App-C32\UDP.o
LCDText             0x21              ..\Microchip\TCPIP Stack\Objects - TCPIP Demo App-C32\LCDBlocking.o
curHTTP             0x8c              ..\Microchip\TCPIP Stack\Objects - TCPIP Demo App-C32\HTTP2.o
bufWeight           0x32              Objects - TCPIP Demo App-C32\CustomHTTPApp.o
activeUDPSocket     0x1               ..\Microchip\TCPIP Stack\Objects - TCPIP Demo App-C32\UDP.o
curHTTPID           0x1               ..\Microchip\TCPIP Stack\Objects - TCPIP Demo App-C32\HTTP2.o
remoteNode          0xa               ..\Microchip\TCPIP Stack\Objects - TCPIP Demo App-C32\StackTsk.o
DDNSClient          0x20              ..\Microchip\TCPIP Stack\Objects - TCPIP Demo App-C32\DynDNS.o
SMTPClient          0x2c              ..\Microchip\TCPIP Stack\Objects - TCPIP Demo App-C32\SMTP.o
bufHeight           0x32              Objects - TCPIP Demo App-C32\CustomHTTPApp.o
lastBlock           0x40              ..\Microchip\TCPIP Stack\Objects - TCPIP Demo App-C32\Hashes.o
AppConfig           0x33              Objects - TCPIP Demo App-C32\MainDemo.o
bufName             0x32              Objects - TCPIP Demo App-C32\CustomHTTPApp.o
bufEye              0x32              Objects - TCPIP Demo App-C32\CustomHTTPApp.o
UDPRxCount          0x2               ..\Microchip\TCPIP Stack\Objects - TCPIP Demo App-C32\UDP.o
UDPSocketInfo       0x8c              ..\Microchip\TCPIP Stack\Objects - TCPIP Demo App-C32\UDP.o
httpStubs           0x10              ..\Microchip\TCPIP Stack\Objects - TCPIP Demo App-C32\HTTP2.o
AN0String           0x8               Objects - TCPIP Demo App-C32\MainDemo.o
bufGender           0x32              Objects - TCPIP Demo App-C32\CustomHTTPApp.o

Microchip PIC32 Memory-Usage Report

kseg0 Program-Memory Usage
section                    address  length [bytes]      (dec)  Description
-------                 ----------  -------------------------  -----------
.text                   0x9d000000        0x1c9e0      117216  Application's executable code 
.rodata                 0x9d01c9e0          0xf1c        3868  Read-only constant data 
.eh_frame               0x9d01d8fc           0x20          32  Stack unwind info 
.data                   0x9d01d91c          0x23c         572  Data-initialization template 
.sdata                  0x9d01db58           0x28          40  Small data-initialization template 
      Total kseg0_program_mem used  :     0x1db80      121728  23.2% of 0x80000

kseg0 Boot-Memory Usage
section                    address  length [bytes]      (dec)  Description
-------                 ----------  -------------------------  -----------
.startup                0x9fc00490          0x1e0         480  C startup code 
         Total kseg0_boot_mem used  :       0x1e0         480  19.9% of 0x970

Exception-Memory Usage 
section                    address  length [bytes]      (dec)  Description
-------                 ----------  -------------------------  -----------
.app_excpt              0x9fc01180           0x10          16  General-Exception handler 
.vector_4               0x9fc01280            0x8           8  Interrupt Vector 4 
          Total exception_mem used  :        0x18          24  0.6% of 0x1000

kseg1 Boot-Memory Usage
section                    address  length [bytes]      (dec)  Description
-------                 ----------  -------------------------  -----------
.reset                  0xbfc00000           0x10          16  Reset handler 
.bev_excpt              0xbfc00380           0x10          16  BEV-Exception handler 
         Total kseg1_boot_mem used  :        0x20          32  2.7% of 0x490
        --------------------------------------------------------------------------
         Total Program Memory used  :     0x1dd98      122264  23.0% of 0x81e00
        --------------------------------------------------------------------------


kseg1 Data-Memory Usage
section                    address  length [bytes]      (dec)  Description
-------                 ----------  -------------------------  -----------
.data                   0xa0000000          0x23c         572  Initialized data 
.sdata                  0xa000023c           0x28          40  Small initialized data 
.sbss                   0xa0000264          0x110         272  Small uninitialized data 
.bss                    0xa0000374          0x6f8        1784  Uninitialized data 
.stack                  0xa0000a6c          0x400        1024  Minimum space reserved for stack 
         Total kseg1_data_mem used  :       0xe6c        3692  11.3% of 0x8000
        --------------------------------------------------------------------------
            Total Data Memory used  :       0xe6c        3692  11.3% of 0x8000
        --------------------------------------------------------------------------

Memory Configuration

Name             Origin             Length             Attributes
kseg0_program_mem 0x9d000000         0x00080000         xr
kseg0_boot_mem   0x9fc00490         0x00000970
exception_mem    0x9fc01000         0x00001000
kseg1_boot_mem   0xbfc00000         0x00000490
debug_exec_mem   0xbfc02000         0x00000ff0
config3          0xbfc02ff0         0x00000004
config2          0xbfc02ff4         0x00000004
config1          0xbfc02ff8         0x00000004
config0          0xbfc02ffc         0x00000004
kseg1_data_mem   0xa0000000         0x00008000         w !x
sfrs             0xbf800000         0x00100000
*default*        0x00000000         0xffffffff

Linker script and memory map

LOAD C:/Program Files/Microchip/MPLAB C32/bin/../lib/gcc/pic32mx/3.4.4/../../../../pic32mx/lib/size/crt0.o
LOAD Objects - TCPIP Demo App-C32\MainDemo.o
LOAD Objects - TCPIP Demo App-C32\CustomHTTPApp.o
LOAD ..\Microchip\TCPIP Stack\Objects - TCPIP Demo App-C32\UDPPerformanceTest.o
LOAD ..\Microchip\TCPIP Stack\Objects - TCPIP Demo App-C32\Announce.o
LOAD ..\Microchip\TCPIP Stack\Objects - TCPIP Demo App-C32\ARP.o
LOAD ..\Microchip\TCPIP Stack\Objects - TCPIP Demo App-C32\Delay.o
LOAD ..\Microchip\TCPIP Stack\Objects - TCPIP Demo App-C32\DHCP.o
LOAD ..\Microchip\TCPIP Stack\Objects - TCPIP Demo App-C32\DHCPs.o
LOAD ..\Microchip\TCPIP Stack\Objects - TCPIP Demo App-C32\DNS.o
LOAD ..\Microchip\TCPIP Stack\Objects - TCPIP Demo App-C32\DynDNS.o
LOAD ..\Microchip\TCPIP Stack\Objects - TCPIP Demo App-C32\ENC28J60.o
LOAD ..\Microchip\TCPIP Stack\Objects - TCPIP Demo App-C32\FTP.o
LOAD ..\Microchip\TCPIP Stack\Objects - TCPIP Demo App-C32\Hashes.o
LOAD ..\Microchip\TCPIP Stack\Objects - TCPIP Demo App-C32\Helpers.o
LOAD ..\Microchip\TCPIP Stack\Objects - TCPIP Demo App-C32\HTTP2.o
LOAD ..\Microchip\TCPIP Stack\Objects - TCPIP Demo App-C32\HTTP.o
LOAD ..\Microchip\TCPIP Stack\Objects - TCPIP Demo App-C32\ICMP.o
LOAD ..\Microchip\TCPIP Stack\Objects - TCPIP Demo App-C32\IP.o
LOAD ..\Microchip\TCPIP Stack\Objects - TCPIP Demo App-C32\LCDBlocking.o
LOAD ..\Microchip\TCPIP Stack\Objects - TCPIP Demo App-C32\MPFS2.o
LOAD ..\Microchip\TCPIP Stack\Objects - TCPIP Demo App-C32\MPFS.o
LOAD ..\Microchip\TCPIP Stack\Objects - TCPIP Demo App-C32\NBNS.o
LOAD ..\Microchip\TCPIP Stack\Objects - TCPIP Demo App-C32\Reboot.o
LOAD ..\Microchip\TCPIP Stack\Objects - TCPIP Demo App-C32\SMTP.o
LOAD ..\Microchip\TCPIP Stack\Objects - TCPIP Demo App-C32\SNMP.o
LOAD ..\Microchip\TCPIP Stack\Objects - TCPIP Demo App-C32\SNTP.o
LOAD ..\Microchip\TCPIP Stack\Objects - TCPIP Demo App-C32\SPIEEPROM.o
LOAD ..\Microchip\TCPIP Stack\Objects - TCPIP Demo App-C32\SPIFlash.o
LOAD ..\Microchip\TCPIP Stack\Objects - TCPIP Demo App-C32\SPIRAM.o
LOAD ..\Microchip\TCPIP Stack\Objects - TCPIP Demo App-C32\StackTsk.o
LOAD ..\Microchip\TCPIP Stack\Objects - TCPIP Demo App-C32\TCP.o
LOAD ..\Microchip\TCPIP Stack\Objects - TCPIP Demo App-C32\TCPPerformanceTest.o
LOAD ..\Microchip\TCPIP Stack\Objects - TCPIP Demo App-C32\Telnet.o
LOAD ..\Microchip\TCPIP Stack\Objects - TCPIP Demo App-C32\TFTPc.o
LOAD ..\Microchip\TCPIP Stack\Objects - TCPIP Demo App-C32\Tick.o
LOAD ..\Microchip\TCPIP Stack\Objects - TCPIP Demo App-C32\UART2TCPBridge.o
LOAD ..\Microchip\TCPIP Stack\Objects - TCPIP Demo App-C32\UART.o
LOAD ..\Microchip\TCPIP Stack\Objects - TCPIP Demo App-C32\UDP.o
LOAD Objects - TCPIP Demo App-C32\CustomSNMPApp.o
LOAD Objects - TCPIP Demo App-C32\UARTConfig.o
LOAD Objects - TCPIP Demo App-C32\GenericTCPClient.o
LOAD Objects - TCPIP Demo App-C32\GenericTCPServer.o
LOAD Objects - TCPIP Demo App-C32\LegacyHTTPApp.o
LOAD Objects - TCPIP Demo App-C32\PingDemo.o
LOAD Objects - TCPIP Demo App-C32\SMTPDemo.o
LOAD ..\Microchip\TCPIP Stack\Objects - TCPIP Demo App-C32\BerkeleyAPI.o
LOAD Objects - TCPIP Demo App-C32\BerkeleyUDPClientDemo.o
LOAD Objects - TCPIP Demo App-C32\BerkeleyTCPClientDemo.o
LOAD Objects - TCPIP Demo App-C32\BerkeleyTCPServerDemo.o
LOAD ..\Microchip\TCPIP Stack\Objects - TCPIP Demo App-C32\ENCX24J600.o
LOAD ..\Microchip\TCPIP Stack\Objects - TCPIP Demo App-C32\Random.o
LOAD ..\Microchip\TCPIP Stack\Objects - TCPIP Demo App-C32\RSA.o
LOAD ..\Microchip\TCPIP Stack\Objects - TCPIP Demo App-C32\SSL.o
LOAD ..\Microchip\TCPIP Stack\Objects - TCPIP Demo App-C32\ARCFOUR.o
LOAD ..\Microchip\TCPIP Stack\Objects - TCPIP Demo App-C32\BigInt.o
LOAD ..\Microchip\TCPIP Stack\Objects - TCPIP Demo App-C32\BigInt_helper_C32.o
LOAD Objects - TCPIP Demo App-C32\CustomSSLCert.o
LOAD Objects - TCPIP Demo App-C32\MPFSImg2-C32.o
                0x00000001                __MPLAB_BUILD = 0x1
LOAD C:/Program Files/Microchip/MPLAB C32/bin/../lib/gcc/pic32mx/3.4.4/size\libgcc.a
START GROUP
LOAD C:/Program Files/Microchip/MPLAB C32/bin/../lib/gcc/pic32mx/3.4.4/../../../../pic32mx/lib/size\libc.a
LOAD C:/Program Files/Microchip/MPLAB C32/bin/../lib/gcc/pic32mx/3.4.4/../../../../pic32mx/lib/size\libm.a
LOAD C:/Program Files/Microchip/MPLAB C32/bin/../lib/gcc/pic32mx/3.4.4/../../../../pic32mx/lib/size\libe.a
LOAD C:/Program Files/Microchip/MPLAB C32/bin/../lib/gcc/pic32mx/3.4.4/../../../../pic32mx/lib/size\libdsp.a
LOAD C:/Program Files/Microchip/MPLAB C32/bin/../lib/gcc/pic32mx/3.4.4/../../../../pic32mx/lib/size\libmchp_peripheral.a
LOAD C:/Program Files/Microchip/MPLAB C32/bin/../lib/gcc/pic32mx/3.4.4/../../../../pic32mx/lib/size\libmchp_peripheral_32MX360F512L.a
END GROUP
LOAD C:/Program Files/Microchip/MPLAB C32/bin/../lib/gcc/pic32mx/3.4.4/size\libgcc.a
                0x00000400                PROVIDE (_min_stack_size, 0x400)
                0x00000000                PROVIDE (_min_heap_size, 0x0)
LOAD C:/Program Files/Microchip/MPLAB C32/bin/../lib/gcc/pic32mx/3.4.4/../../../../pic32mx/lib/./proc/32MX360F512L\processor.o
                0x00000001                PROVIDE (_vector_spacing, 0x1)
                0x9fc01000                _ebase_address = 0x9fc01000
                0xbfc00000                _RESET_ADDR = 0xbfc00000
                0xbfc00380                _BEV_EXCPT_ADDR = 0xbfc00380
                0xbfc00480                _DBG_EXCPT_ADDR = 0xbfc00480
                0xbfc02000                _DBG_CODE_ADDR = 0xbfc02000
                0x9fc01180                _GEN_EXCPT_ADDR = (_ebase_address + 0x180)

.config_BFC02FF0
 *(.config_BFC02FF0)

.config_BFC02FF4
                0xbfc02ff4        0x4
 *(.config_BFC02FF4)
 .config_BFC02FF4
                0xbfc02ff4        0x4 Objects - TCPIP Demo App-C32\MainDemo.o

.config_BFC02FF8
                0xbfc02ff8        0x4
 *(.config_BFC02FF8)
 .config_BFC02FF8
                0xbfc02ff8        0x4 Objects - TCPIP Demo App-C32\MainDemo.o

.config_BFC02FFC
                0xbfc02ffc        0x4
 *(.config_BFC02FFC)
 .config_BFC02FFC
                0xbfc02ffc        0x4 Objects - TCPIP Demo App-C32\MainDemo.o

.reset          0xbfc00000       0x10
 *(.reset)
 .reset         0xbfc00000       0x10 C:/Program Files/Microchip/MPLAB C32/bin/../lib/gcc/pic32mx/3.4.4/../../../../pic32mx/lib/size/crt0.o
                0xbfc00000                _reset

.bev_excpt      0xbfc00380       0x10
 *(.bev_handler)
 .bev_handler   0xbfc00380       0x10 C:/Program Files/Microchip/MPLAB C32/bin/../lib/gcc/pic32mx/3.4.4/../../../../pic32mx/lib/size/crt0.o

.dbg_excpt      0xbfc00480        0x0
                0xbfc00480                . = (. + DEFINED (_DEBUGGER)?0x8:0x0)

.dbg_code       0xbfc02000        0x0
                0xbfc02000                . = (. + DEFINED (_DEBUGGER)?0xff0:0x0)

.app_excpt      0x9fc01180       0x10
 *(.gen_handler)
 .gen_handler   0x9fc01180       0x10 C:/Program Files/Microchip/MPLAB C32/bin/../lib/gcc/pic32mx/3.4.4/../../../../pic32mx/lib/size/crt0.o

.vector_0       0x9fc01200        0x0
 *(.vector_0)
                0x00000001                ASSERT (((_vector_spacing == 0x0) || (SIZEOF (.vector_0) <= (_vector_spacing << 0x5))), function at exception vector 0 too large)

.vector_1       0x9fc01220        0x0
 *(.vector_1)
                0x00000001                ASSERT (((_vector_spacing == 0x0) || (SIZEOF (.vector_1) <= (_vector_spacing << 0x5))), function at exception vector 1 too large)

.vector_2       0x9fc01240        0x0
 *(.vector_2)
                0x00000001                ASSERT (((_vector_spacing == 0x0) || (SIZEOF (.vector_2) <= (_vector_spacing << 0x5))), function at exception vector 2 too large)

.vector_3       0x9fc01260        0x0
 *(.vector_3)
                0x00000001                ASSERT (((_vector_spacing == 0x0) || (SIZEOF (.vector_3) <= (_vector_spacing << 0x5))), function at exception vector 3 too large)

.vector_4       0x9fc01280        0x8
 *(.vector_4)
 .vector_4      0x9fc01280        0x8 ..\Microchip\TCPIP Stack\Objects - TCPIP Demo App-C32\Tick.o
                0x00000001                ASSERT (((_vector_spacing == 0x0) || (SIZEOF (.vector_4) <= (_vector_spacing << 0x5))), function at exception vector 4 too large)

.vector_5       0x9fc012a0        0x0
 *(.vector_5)
                0x00000001                ASSERT (((_vector_spacing == 0x0) || (SIZEOF (.vector_5) <= (_vector_spacing << 0x5))), function at exception vector 5 too large)

.vector_6       0x9fc012c0        0x0
 *(.vector_6)
                0x00000001                ASSERT (((_vector_spacing == 0x0) || (SIZEOF (.vector_6) <= (_vector_spacing << 0x5))), function at exception vector 6 too large)

.vector_7       0x9fc012e0        0x0
 *(.vector_7)
                0x00000001                ASSERT (((_vector_spacing == 0x0) || (SIZEOF (.vector_7) <= (_vector_spacing << 0x5))), function at exception vector 7 too large)

.vector_8       0x9fc01300        0x0
 *(.vector_8)
                0x00000001                ASSERT (((_vector_spacing == 0x0) || (SIZEOF (.vector_8) <= (_vector_spacing << 0x5))), function at exception vector 8 too large)

.vector_9       0x9fc01320        0x0
 *(.vector_9)
                0x00000001                ASSERT (((_vector_spacing == 0x0) || (SIZEOF (.vector_9) <= (_vector_spacing << 0x5))), function at exception vector 9 too large)

.vector_10      0x9fc01340        0x0
 *(.vector_10)
                0x00000001                ASSERT (((_vector_spacing == 0x0) || (SIZEOF (.vector_10) <= (_vector_spacing << 0x5))), function at exception vector 10 too large)

.vector_11      0x9fc01360        0x0
 *(.vector_11)
                0x00000001                ASSERT (((_vector_spacing == 0x0) || (SIZEOF (.vector_11) <= (_vector_spacing << 0x5))), function at exception vector 11 too large)

.vector_12      0x9fc01380        0x0
 *(.vector_12)
                0x00000001                ASSERT (((_vector_spacing == 0x0) || (SIZEOF (.vector_12) <= (_vector_spacing << 0x5))), function at exception vector 12 too large)

.vector_13      0x9fc013a0        0x0
 *(.vector_13)
                0x00000001                ASSERT (((_vector_spacing == 0x0) || (SIZEOF (.vector_13) <= (_vector_spacing << 0x5))), function at exception vector 13 too large)

.vector_14      0x9fc013c0        0x0
 *(.vector_14)
                0x00000001                ASSERT (((_vector_spacing == 0x0) || (SIZEOF (.vector_14) <= (_vector_spacing << 0x5))), function at exception vector 14 too large)

.vector_15      0x9fc013e0        0x0
 *(.vector_15)
                0x00000001                ASSERT (((_vector_spacing == 0x0) || (SIZEOF (.vector_15) <= (_vector_spacing << 0x5))), function at exception vector 15 too large)

.vector_16      0x9fc01400        0x0
 *(.vector_16)
                0x00000001                ASSERT (((_vector_spacing == 0x0) || (SIZEOF (.vector_16) <= (_vector_spacing << 0x5))), function at exception vector 16 too large)

.vector_17      0x9fc01420        0x0
 *(.vector_17)
                0x00000001                ASSERT (((_vector_spacing == 0x0) || (SIZEOF (.vector_17) <= (_vector_spacing << 0x5))), function at exception vector 17 too large)

.vector_18      0x9fc01440        0x0
 *(.vector_18)
                0x00000001                ASSERT (((_vector_spacing == 0x0) || (SIZEOF (.vector_18) <= (_vector_spacing << 0x5))), function at exception vector 18 too large)

.vector_19      0x9fc01460        0x0
 *(.vector_19)
                0x00000001                ASSERT (((_vector_spacing == 0x0) || (SIZEOF (.vector_19) <= (_vector_spacing << 0x5))), function at exception vector 19 too large)

.vector_20      0x9fc01480        0x0
 *(.vector_20)
                0x00000001                ASSERT (((_vector_spacing == 0x0) || (SIZEOF (.vector_20) <= (_vector_spacing << 0x5))), function at exception vector 20 too large)

.vector_21      0x9fc014a0        0x0
 *(.vector_21)
                0x00000001                ASSERT (((_vector_spacing == 0x0) || (SIZEOF (.vector_21) <= (_vector_spacing << 0x5))), function at exception vector 21 too large)

.vector_22      0x9fc014c0        0x0
 *(.vector_22)
                0x00000001                ASSERT (((_vector_spacing == 0x0) || (SIZEOF (.vector_22) <= (_vector_spacing << 0x5))), function at exception vector 22 too large)

.vector_23      0x9fc014e0        0x0
 *(.vector_23)
                0x00000001                ASSERT (((_vector_spacing == 0x0) || (SIZEOF (.vector_23) <= (_vector_spacing << 0x5))), function at exception vector 23 too large)

.vector_24      0x9fc01500        0x0
 *(.vector_24)
                0x00000001                ASSERT (((_vector_spacing == 0x0) || (SIZEOF (.vector_24) <= (_vector_spacing << 0x5))), function at exception vector 24 too large)

.vector_25      0x9fc01520        0x0
 *(.vector_25)
                0x00000001                ASSERT (((_vector_spacing == 0x0) || (SIZEOF (.vector_25) <= (_vector_spacing << 0x5))), function at exception vector 25 too large)

.vector_26      0x9fc01540        0x0
 *(.vector_26)
                0x00000001                ASSERT (((_vector_spacing == 0x0) || (SIZEOF (.vector_26) <= (_vector_spacing << 0x5))), function at exception vector 26 too large)

.vector_27      0x9fc01560        0x0
 *(.vector_27)
                0x00000001                ASSERT (((_vector_spacing == 0x0) || (SIZEOF (.vector_27) <= (_vector_spacing << 0x5))), function at exception vector 27 too large)

.vector_28      0x9fc01580        0x0
 *(.vector_28)
                0x00000001                ASSERT (((_vector_spacing == 0x0) || (SIZEOF (.vector_28) <= (_vector_spacing << 0x5))), function at exception vector 28 too large)

.vector_29      0x9fc015a0        0x0
 *(.vector_29)
                0x00000001                ASSERT (((_vector_spacing == 0x0) || (SIZEOF (.vector_29) <= (_vector_spacing << 0x5))), function at exception vector 29 too large)

.vector_30      0x9fc015c0        0x0
 *(.vector_30)
                0x00000001                ASSERT (((_vector_spacing == 0x0) || (SIZEOF (.vector_30) <= (_vector_spacing << 0x5))), function at exception vector 30 too large)

.vector_31      0x9fc015e0        0x0
 *(.vector_31)
                0x00000001                ASSERT (((_vector_spacing == 0x0) || (SIZEOF (.vector_31) <= (_vector_spacing << 0x5))), function at exception vector 31 too large)

.vector_32      0x9fc01600        0x0
 *(.vector_32)
                0x00000001                ASSERT (((_vector_spacing == 0x0) || (SIZEOF (.vector_32) <= (_vector_spacing << 0x5))), function at exception vector 32 too large)

.vector_33      0x9fc01620        0x0
 *(.vector_33)
                0x00000001                ASSERT (((_vector_spacing == 0x0) || (SIZEOF (.vector_33) <= (_vector_spacing << 0x5))), function at exception vector 33 too large)

.vector_34      0x9fc01640        0x0
 *(.vector_34)
                0x00000001                ASSERT (((_vector_spacing == 0x0) || (SIZEOF (.vector_34) <= (_vector_spacing << 0x5))), function at exception vector 34 too large)

.vector_35      0x9fc01660        0x0
 *(.vector_35)
                0x00000001                ASSERT (((_vector_spacing == 0x0) || (SIZEOF (.vector_35) <= (_vector_spacing << 0x5))), function at exception vector 35 too large)

.vector_36      0x9fc01680        0x0
 *(.vector_36)
                0x00000001                ASSERT (((_vector_spacing == 0x0) || (SIZEOF (.vector_36) <= (_vector_spacing << 0x5))), function at exception vector 36 too large)

.vector_37      0x9fc016a0        0x0
 *(.vector_37)
                0x00000001                ASSERT (((_vector_spacing == 0x0) || (SIZEOF (.vector_37) <= (_vector_spacing << 0x5))), function at exception vector 37 too large)

.vector_38      0x9fc016c0        0x0
 *(.vector_38)
                0x00000001                ASSERT (((_vector_spacing == 0x0) || (SIZEOF (.vector_38) <= (_vector_spacing << 0x5))), function at exception vector 38 too large)

.vector_39      0x9fc016e0        0x0
 *(.vector_39)
                0x00000001                ASSERT (((_vector_spacing == 0x0) || (SIZEOF (.vector_39) <= (_vector_spacing << 0x5))), function at exception vector 39 too large)

.vector_40      0x9fc01700        0x0
 *(.vector_40)
                0x00000001                ASSERT (((_vector_spacing == 0x0) || (SIZEOF (.vector_40) <= (_vector_spacing << 0x5))), function at exception vector 40 too large)

.vector_41      0x9fc01720        0x0
 *(.vector_41)
                0x00000001                ASSERT (((_vector_spacing == 0x0) || (SIZEOF (.vector_41) <= (_vector_spacing << 0x5))), function at exception vector 41 too large)

.vector_42      0x9fc01740        0x0
 *(.vector_42)
                0x00000001                ASSERT (((_vector_spacing == 0x0) || (SIZEOF (.vector_42) <= (_vector_spacing << 0x5))), function at exception vector 42 too large)

.vector_43      0x9fc01760        0x0
 *(.vector_43)
                0x00000001                ASSERT (((_vector_spacing == 0x0) || (SIZEOF (.vector_43) <= (_vector_spacing << 0x5))), function at exception vector 43 too large)

.vector_44      0x9fc01780        0x0
 *(.vector_44)
                0x00000001                ASSERT (((_vector_spacing == 0x0) || (SIZEOF (.vector_44) <= (_vector_spacing << 0x5))), function at exception vector 44 too large)

.vector_45      0x9fc017a0        0x0
 *(.vector_45)
                0x00000001                ASSERT (((_vector_spacing == 0x0) || (SIZEOF (.vector_45) <= (_vector_spacing << 0x5))), function at exception vector 45 too large)

.vector_46      0x9fc017c0        0x0
 *(.vector_46)
                0x00000001                ASSERT (((_vector_spacing == 0x0) || (SIZEOF (.vector_46) <= (_vector_spacing << 0x5))), function at exception vector 46 too large)

.vector_47      0x9fc017e0        0x0
 *(.vector_47)
                0x00000001                ASSERT (((_vector_spacing == 0x0) || (SIZEOF (.vector_47) <= (_vector_spacing << 0x5))), function at exception vector 47 too large)

.vector_48      0x9fc01800        0x0
 *(.vector_48)
                0x00000001                ASSERT (((_vector_spacing == 0x0) || (SIZEOF (.vector_48) <= (_vector_spacing << 0x5))), function at exception vector 48 too large)

.vector_49      0x9fc01820        0x0
 *(.vector_49)
                0x00000001                ASSERT (((_vector_spacing == 0x0) || (SIZEOF (.vector_49) <= (_vector_spacing << 0x5))), function at exception vector 49 too large)

.vector_50      0x9fc01840        0x0
 *(.vector_50)
                0x00000001                ASSERT (((_vector_spacing == 0x0) || (SIZEOF (.vector_50) <= (_vector_spacing << 0x5))), function at exception vector 50 too large)

.vector_51      0x9fc01860        0x0
 *(.vector_51)
                0x00000001                ASSERT (((_vector_spacing == 0x0) || (SIZEOF (.vector_51) <= (_vector_spacing << 0x5))), function at exception vector 51 too large)

.vector_52      0x9fc01880        0x0
 *(.vector_52)
                0x00000001                ASSERT (((_vector_spacing == 0x0) || (SIZEOF (.vector_52) <= (_vector_spacing << 0x5))), function at exception vector 52 too large)

.vector_53      0x9fc018a0        0x0
 *(.vector_53)
                0x00000001                ASSERT (((_vector_spacing == 0x0) || (SIZEOF (.vector_53) <= (_vector_spacing << 0x5))), function at exception vector 53 too large)

.vector_54      0x9fc018c0        0x0
 *(.vector_54)
                0x00000001                ASSERT (((_vector_spacing == 0x0) || (SIZEOF (.vector_54) <= (_vector_spacing << 0x5))), function at exception vector 54 too large)

.vector_55      0x9fc018e0        0x0
 *(.vector_55)
                0x00000001                ASSERT (((_vector_spacing == 0x0) || (SIZEOF (.vector_55) <= (_vector_spacing << 0x5))), function at exception vector 55 too large)

.vector_56      0x9fc01900        0x0
 *(.vector_56)
                0x00000001                ASSERT (((_vector_spacing == 0x0) || (SIZEOF (.vector_56) <= (_vector_spacing << 0x5))), function at exception vector 56 too large)

.vector_57      0x9fc01920        0x0
 *(.vector_57)
                0x00000001                ASSERT (((_vector_spacing == 0x0) || (SIZEOF (.vector_57) <= (_vector_spacing << 0x5))), function at exception vector 57 too large)

.vector_58      0x9fc01940        0x0
 *(.vector_58)
                0x00000001                ASSERT (((_vector_spacing == 0x0) || (SIZEOF (.vector_58) <= (_vector_spacing << 0x5))), function at exception vector 58 too large)

.vector_59      0x9fc01960        0x0
 *(.vector_59)
                0x00000001                ASSERT (((_vector_spacing == 0x0) || (SIZEOF (.vector_59) <= (_vector_spacing << 0x5))), function at exception vector 59 too large)

.vector_60      0x9fc01980        0x0
 *(.vector_60)
                0x00000001                ASSERT (((_vector_spacing == 0x0) || (SIZEOF (.vector_60) <= (_vector_spacing << 0x5))), function at exception vector 60 too large)

.vector_61      0x9fc019a0        0x0
 *(.vector_61)
                0x00000001                ASSERT (((_vector_spacing == 0x0) || (SIZEOF (.vector_61) <= (_vector_spacing << 0x5))), function at exception vector 61 too large)

.vector_62      0x9fc019c0        0x0
 *(.vector_62)
                0x00000001                ASSERT (((_vector_spacing == 0x0) || (SIZEOF (.vector_62) <= (_vector_spacing << 0x5))), function at exception vector 62 too large)

.vector_63      0x9fc019e0        0x0
 *(.vector_63)
                0x00000001                ASSERT (((_vector_spacing == 0x0) || (SIZEOF (.vector_63) <= (_vector_spacing << 0x5))), function at exception vector 63 too large)

.startup        0x9fc00490      0x1e0
 *(.startup)
 .startup       0x9fc00490      0x1e0 C:/Program Files/Microchip/MPLAB C32/bin/../lib/gcc/pic32mx/3.4.4/../../../../pic32mx/lib/size/crt0.o

.text           0x9d000000    0x1c9e0
                0x9d000000                _text_begin = .
 *(.text .stub .text.* .gnu.linkonce.t.*)
 .text          0x9d000000       0x18 C:/Program Files/Microchip/MPLAB C32/bin/../lib/gcc/pic32mx/3.4.4/../../../../pic32mx/lib/size/crt0.o
 .text          0x9d000018      0xb34 Objects - TCPIP Demo App-C32\MainDemo.o
                0x9d000044                main
                0x9d00016c                DisplayIPValue
                0x9d000018                _general_exception_handler
 .text          0x9d000b4c      0x844 Objects - TCPIP Demo App-C32\CustomHTTPApp.o
                0x9d000b4c                HTTPNeedsAuth
                0x9d000fc4                HTTPExecutePost
                0x9d000bdc                HTTPCheckAuth
                0x9d000c5c                HTTPExecuteGet
 .text          0x9d001390      0x5ec ..\Microchip\TCPIP Stack\Objects - TCPIP Demo App-C32\ARP.o
                0x9d0017f4                ARPIsResolved
                0x9d001524                ARPProcess
                0x9d001494                ARPInit
                0x9d001714                ARPResolve
 .text          0x9d00197c       0xec ..\Microchip\TCPIP Stack\Objects - TCPIP Demo App-C32\Delay.o
                0x9d00197c                DelayMs
                0x9d001a00                Delay10us
 .text          0x9d001a68     0x11d4 ..\Microchip\TCPIP Stack\Objects - TCPIP Demo App-C32\DHCP.o
                0x9d001a68                DHCPReset
                0x9d001ba0                DHCPTask
                0x9d001ad8                DHCPDisable
                0x9d001b44                DHCPEnable
 .text          0x9d002c3c      0xae0 ..\Microchip\TCPIP Stack\Objects - TCPIP Demo App-C32\DHCPs.o
                0x9d002c3c                DHCPServerTask
 .text          0x9d00371c      0xe9c ..\Microchip\TCPIP Stack\Objects - TCPIP Demo App-C32\DNS.o
                0x9d003774                DNSEndUsage
                0x9d0037e8                DNSResolve
                0x9d00387c                DNSIsResolved
                0x9d00371c                DNSBeginUsage
 .text          0x9d0045b8     0x1788 ..\Microchip\TCPIP Stack\Objects - TCPIP Demo App-C32\DynDNS.o
                0x9d005cec                DDNSGetLastIP
                0x9d005c6c                DDNSSetService
                0x9d004658                DDNSTask
                0x9d0045b8                DDNSInit
                0x9d005d1c                DDNSGetLastStatus
                0x9d005c28                DDNSForceUpdate
 .text          0x9d005d40     0x24f8 ..\Microchip\TCPIP Stack\Objects - TCPIP Demo App-C32\ENC28J60.o
                0x9d0060d4                MACIsTxReady
                0x9d006d94                MACMemCopyAsync
                0x9d00761c                MACPutArray
                0x9d006944                MACSetReadPtrInRx
                0x9d005d40                MACInit
                0x9d006bfc                CalcIPBufferChecksum
                0x9d006348                MACGetHeader
                0x9d006120                MACDiscardRx
                0x9d006af4                MACCalcRxChecksum
                0x9d007f4c                WritePHYReg
                0x9d00817c                SetCLKOUT
                0x9d008064                MACPowerDown
                0x9d00661c                MACFlush
                0x9d0069cc                MACSetWritePtr
                0x9d0071d4                MACIsMemCopyDone
                0x9d008108                MACPowerUp
                0x9d007560                MACPut
                0x9d006094                MACIsLinked
                0x9d0072d4                MACGetArray
                0x9d007220                MACGet
                0x9d0081d8                GetCLKOUT
                0x9d006a60                MACSetReadPtr
                0x9d0061c0                MACGetFreeRxSize
                0x9d007b88                ReadPHYReg
                0x9d006530                MACPutHeader
 .text          0x9d008238      0x76c ..\Microchip\TCPIP Stack\Objects - TCPIP Demo App-C32\Hashes.o
                0x9d0086c8                MD5Calculate
                0x9d008238                HashAddData
                0x9d008298                MD5Initialize
                0x9d00830c                MD5AddData
 .text          0x9d0089a4     0x13b4 ..\Microchip\TCPIP Stack\Objects - TCPIP Demo App-C32\Helpers.o
                0x9d0094e0                uitoa
                0x9d009aa8                swapl
                0x9d0097fc                btohexa_high
                0x9d009a5c                swaps
                0x9d008bec                StringToIPAddress
                0x9d009ca0                FormatNetBIOSName
                0x9d00986c                btohexa_low
                0x9d009b30                CalcIPChecksum
                0x9d009728                hexatob
                0x9d0098dc                stricmppgm2ram
                0x9d008eec                Base64Decode
                0x9d009604                ultoa
                0x9d009c10                strupr
                0x9d0089a4                GenerateRandomDWORD
                0x9d009250                Base64Encode
 .text          0x9d009d58     0x3234 ..\Microchip\TCPIP Stack\Objects - TCPIP Demo App-C32\HTTP2.o
                0x9d009d58                HTTPPrint
                0x9d00c8e0                HTTPReadPostName
                0x9d009db4                HTTPPrint_
                0x9d00c95c                HTTPReadPostValue
                0x9d00c640                HTTPURLDecode
                0x9d009f0c                HTTPServer
                0x9d00cd8c                HTTPIncFile
                0x9d009e04                HTTPInit
                0x9d00c814                HTTPGetArg
 .text          0x9d00cf8c      0x148 ..\Microchip\TCPIP Stack\Objects - TCPIP Demo App-C32\ICMP.o
                0x9d00cf8c                ICMPProcess
 .text          0x9d00d0d4      0x31c ..\Microchip\TCPIP Stack\Objects - TCPIP Demo App-C32\IP.o
                0x9d00d0d4                IPGetHeader
                0x9d00d210                IPPutHeader
                0x9d00d31c                IPSetRxBuffer
 .text          0x9d00d3f0      0x48c ..\Microchip\TCPIP Stack\Objects - TCPIP Demo App-C32\LCDBlocking.o
                0x9d00d4cc                LCDInit
                0x9d00d820                LCDErase
                0x9d00d64c                LCDUpdate
 .text          0x9d00d87c     0x1818 ..\Microchip\TCPIP Stack\Objects - TCPIP Demo App-C32\MPFS2.o
                0x9d00d87c                MPFSInit
                0x9d00dc3c                MPFSOpenID
                0x9d00ebc0                MPFSGetBytesRem
                0x9d00ea28                MPFSGetFlags
                0x9d00e390                MPFSSeek
                0x9d00ee20                MPFSGetFilename
                0x9d00e088                MPFSGetArray
                0x9d00de3c                MPFSGet
                0x9d00ef30                MPFSGetPosition
                0x9d00eaf4                MPFSGetSize
                0x9d00d904                MPFSOpen
                0x9d00e890                MPFSGetTimestamp
                0x9d00efa4                MPFSGetID
                0x9d00ec6c                MPFSGetStartAddr
                0x9d00ddd0                MPFSClose
                0x9d00e95c                MPFSGetMicrotime
                0x9d00ed3c                MPFSGetEndAddr
                0x9d00e33c                MPFSGetLong
 .text          0x9d00f094      0x6fc ..\Microchip\TCPIP Stack\Objects - TCPIP Demo App-C32\NBNS.o
                0x9d00f094                NBNSTask
 .text          0x9d00f790     0x25c8 ..\Microchip\TCPIP Stack\Objects - TCPIP Demo App-C32\SMTP.o
                0x9d011624                SMTPSendMail
                0x9d011918                SMTPPutString
                0x9d011678                SMTPIsPutReady
                0x9d00f8f8                SMTPTask
                0x9d00f82c                SMTPEndUsage
                0x9d00f790                SMTPBeginUsage
                0x9d011878                SMTPPutArray
                0x9d0119a4                SMTPFlush
                0x9d0116d4                SMTPPut
                0x9d0119dc                SMTPPutDone
                0x9d011650                SMTPIsBusy
 .text          0x9d011d58      0x3c0 ..\Microchip\TCPIP Stack\Objects - TCPIP Demo App-C32\StackTsk.o
                0x9d011e04                StackTask
                0x9d011d58                StackInit
                0x9d0120c8                StackApplications
 .text          0x9d012118     0x8134 ..\Microchip\TCPIP Stack\Objects - TCPIP Demo App-C32\TCP.o
                0x9d0137b8                TCPGetTxFIFOFull
                0x9d01254c                TCPOpen
                0x9d013914                TCPIsGetReady
                0x9d012d88                TCPIsPutReady
                0x9d012c84                TCPGetRemoteInfo
                0x9d012a5c                TCPIsConnected
                0x9d0147e4                TCPFindEx
                0x9d012d00                TCPFlush
                0x9d013ab0                TCPGet
                0x9d015878                TCPProcess
                0x9d012ab8                TCPDisconnect
                0x9d014118                TCPGetRxFIFOFree
                0x9d012f7c                TCPPut
                0x9d0132d0                TCPPutArray
                0x9d013d38                TCPGetArray
                0x9d013754                TCPPutString
                0x9d014858                TCPTick
                0x9d0198f4                TCPAdjustFIFOSize
                0x9d0141c8                TCPFindArrayEx
                0x9d0129b0                TCPWasReset
                0x9d01386c                TCPDiscard
                0x9d01224c                TCPInit
 .text          0x9d01a24c      0x304 ..\Microchip\TCPIP Stack\Objects - TCPIP Demo App-C32\Tick.o
                0x9d01a24c                TickInit
                0x9d01a3cc                TickGetDiv256
                0x9d01a420                TickGetDiv64K
                0x9d01a474                TickConvertToMilliseconds
                0x9d01a398                TickGet
                0x9d01a4cc                _T1Interrupt
 .text          0x9d01a550      0xc90 ..\Microchip\TCPIP Stack\Objects - TCPIP Demo App-C32\UDP.o
                0x9d01acc8                UDPGet
                0x9d01a5bc                UDPTask
                0x9d01aa2c                UDPPutString
                0x9d01ad58                UDPGetArray
                0x9d01a550                UDPInit
                0x9d01a7c4                UDPSetTxBuffer
                0x9d01ac2c                UDPIsGetReady
                0x9d01ae24                UDPDiscard
                0x9d01a814                UDPSetRxBuffer
                0x9d01a5e4                UDPOpen
                0x9d01a864                UDPIsPutReady
                0x9d01aa80                UDPFlush
                0x9d01a8f8                UDPPut
                0x9d01a988                UDPPutArray
                0x9d01a738                UDPClose
                0x9d01ae80                UDPProcess
 .text          0x9d01b1e0      0x2dc Objects - TCPIP Demo App-C32\SMTPDemo.o
                0x9d01b1e0                SMTPDemo
 .text          0x9d01b4bc      0x44c C:/Program Files/Microchip/MPLAB C32/bin/../lib/gcc/pic32mx/3.4.4/size\libgcc.a(_udivdi3.o)
                0x9d01b4bc                __udivdi3
 .text          0x9d01b908       0x98 C:/Program Files/Microchip/MPLAB C32/bin/../lib/gcc/pic32mx/3.4.4/../../../../pic32mx/lib/size\libc.a(memcmp.o)
                0x9d01b908                memcmp
 .text          0x9d01b9a0      0x168 C:/Program Files/Microchip/MPLAB C32/bin/../lib/gcc/pic32mx/3.4.4/../../../../pic32mx/lib/size\libc.a(memcpy.o)
                0x9d01b9a0                memcpy
 .text          0x9d01bb08       0xa8 C:/Program Files/Microchip/MPLAB C32/bin/../lib/gcc/pic32mx/3.4.4/../../../../pic32mx/lib/size\libc.a(memset.o)
                0x9d01bb08                memset
 .text          0x9d01bbb0      0x120 C:/Program Files/Microchip/MPLAB C32/bin/../lib/gcc/pic32mx/3.4.4/../../../../pic32mx/lib/size\libc.a(strcmp.o)
                0x9d01bbb0                strcmp
 .text          0x9d01bcd0      0x1a0 C:/Program Files/Microchip/MPLAB C32/bin/../lib/gcc/pic32mx/3.4.4/../../../../pic32mx/lib/size\libc.a(strcpy.o)
                0x9d01bcd0                strcpy
 .text          0x9d01be70      0x168 C:/Program Files/Microchip/MPLAB C32/bin/../lib/gcc/pic32mx/3.4.4/../../../../pic32mx/lib/size\libc.a(strlen.o)
                0x9d01be70                strlen
 .text.general_exception
                0x9d01bfd8       0xd0 C:/Program Files/Microchip/MPLAB C32/bin/../lib/gcc/pic32mx/3.4.4/../../../../pic32mx/lib/size\libc.a(general-exception.o)
                0x9d01bfd8                _general_exception_context
 .text.strchr   0x9d01c0a8       0x90 C:/Program Files/Microchip/MPLAB C32/bin/../lib/gcc/pic32mx/3.4.4/../../../../pic32mx/lib/size\libc.a(strchr.o)
                0x9d01c0a8                strchr
 .text.strstr   0x9d01c138       0x50 C:/Program Files/Microchip/MPLAB C32/bin/../lib/gcc/pic32mx/3.4.4/../../../../pic32mx/lib/size\libc.a(strstr.o)
                0x9d01c138                strstr
 .text.exit     0x9d01c188       0x9c C:/Program Files/Microchip/MPLAB C32/bin/../lib/gcc/pic32mx/3.4.4/../../../../pic32mx/lib/size\libc.a(exit.o)
                0x9d01c188                exit
 .text.rand_r   0x9d01c224       0x28 C:/Program Files/Microchip/MPLAB C32/bin/../lib/gcc/pic32mx/3.4.4/../../../../pic32mx/lib/size\libc.a(rand.o)
                0x9d01c224                rand_r
 .text.rand     0x9d01c24c       0x4c C:/Program Files/Microchip/MPLAB C32/bin/../lib/gcc/pic32mx/3.4.4/../../../../pic32mx/lib/size\libc.a(rand.o)
                0x9d01c24c                rand
 .text.srand    0x9d01c298       0x44 C:/Program Files/Microchip/MPLAB C32/bin/../lib/gcc/pic32mx/3.4.4/../../../../pic32mx/lib/size\libc.a(rand.o)
                0x9d01c298                srand
 .text.atol     0x9d01c2dc       0x20 C:/Program Files/Microchip/MPLAB C32/bin/../lib/gcc/pic32mx/3.4.4/../../../../pic32mx/lib/size\libc.a(atol.o)
                0x9d01c2dc                atol
 .text.atoi     0x9d01c2fc       0x20 C:/Program Files/Microchip/MPLAB C32/bin/../lib/gcc/pic32mx/3.4.4/../../../../pic32mx/lib/size\libc.a(atoi.o)
                0x9d01c2fc                atoi
 .text.strtol   0x9d01c31c      0x1ec C:/Program Files/Microchip/MPLAB C32/bin/../lib/gcc/pic32mx/3.4.4/../../../../pic32mx/lib/size\libc.a(strtol.o)
                0x9d01c31c                strtol
 .text._filbuf_simple
                0x9d01c508       0x48 C:/Program Files/Microchip/MPLAB C32/bin/../lib/gcc/pic32mx/3.4.4/../../../../pic32mx/lib/size\libc.a(_iobfuncs.o)
                0x9d01c508                _filbuf_simple
 .text._fflush_simple
                0x9d01c550       0x6c C:/Program Files/Microchip/MPLAB C32/bin/../lib/gcc/pic32mx/3.4.4/../../../../pic32mx/lib/size\libc.a(_iobfuncs.o)
                0x9d01c550                _fflush_simple
 .text._flsbuf_simple
                0x9d01c5bc       0xdc C:/Program Files/Microchip/MPLAB C32/bin/../lib/gcc/pic32mx/3.4.4/../../../../pic32mx/lib/size\libc.a(_iobfuncs.o)
                0x9d01c5bc                _flsbuf_simple
 .text._fwrite_simple
                0x9d01c698       0x84 C:/Program Files/Microchip/MPLAB C32/bin/../lib/gcc/pic32mx/3.4.4/../../../../pic32mx/lib/size\libc.a(_iobfuncs.o)
                0x9d01c698                _fwrite_simple
 .text._fsync_simple
                0x9d01c71c       0x34 C:/Program Files/Microchip/MPLAB C32/bin/../lib/gcc/pic32mx/3.4.4/../../../../pic32mx/lib/size\libc.a(_iobfuncs.o)
                0x9d01c71c                _fsync_simple
 .text._weak_pthread_mutex_init
                0x9d01c750        0x8 C:/Program Files/Microchip/MPLAB C32/bin/../lib/gcc/pic32mx/3.4.4/../../../../pic32mx/lib/size\libc.a(stubs.o)
                0x9d01c750                _weak_pthread_mutex_init
                0x9d01c750                pthread_mutex_init
 .text._weak_pthread_mutex_destroy
                0x9d01c758        0x8 C:/Program Files/Microchip/MPLAB C32/bin/../lib/gcc/pic32mx/3.4.4/../../../../pic32mx/lib/size\libc.a(stubs.o)
                0x9d01c758                _weak_pthread_mutex_destroy
                0x9d01c758                pthread_mutex_destroy
 .text._weak_pthread_mutex_lock
                0x9d01c760        0x8 C:/Program Files/Microchip/MPLAB C32/bin/../lib/gcc/pic32mx/3.4.4/../../../../pic32mx/lib/size\libc.a(stubs.o)
                0x9d01c760                _weak_pthread_mutex_lock
                0x9d01c760                pthread_mutex_lock
 .text._weak_pthread_mutex_trylock
                0x9d01c768        0x8 C:/Program Files/Microchip/MPLAB C32/bin/../lib/gcc/pic32mx/3.4.4/../../../../pic32mx/lib/size\libc.a(stubs.o)
                0x9d01c768                _weak_pthread_mutex_trylock
                0x9d01c768                pthread_mutex_trylock
 .text._weak_pthread_mutex_unlock
                0x9d01c770        0x8 C:/Program Files/Microchip/MPLAB C32/bin/../lib/gcc/pic32mx/3.4.4/../../../../pic32mx/lib/size\libc.a(stubs.o)
                0x9d01c770                _weak_pthread_mutex_unlock
                0x9d01c770                pthread_mutex_unlock
 .text._weak_pthread_mutex_setname_np
                0x9d01c778        0x8 C:/Program Files/Microchip/MPLAB C32/bin/../lib/gcc/pic32mx/3.4.4/../../../../pic32mx/lib/size\libc.a(stubs.o)
                0x9d01c778                pthread_mutex_setname_np
                0x9d01c778                _weak_pthread_mutex_setname_np
 .text._weak_pthread_mutexattr_init
                0x9d01c780        0x8 C:/Program Files/Microchip/MPLAB C32/bin/../lib/gcc/pic32mx/3.4.4/../../../../pic32mx/lib/size\libc.a(stubs.o)
                0x9d01c780                _weak_pthread_mutexattr_init
                0x9d01c780                pthread_mutexattr_init
 .text._weak_pthread_mutexattr_destroy
                0x9d01c788        0x8 C:/Program Files/Microchip/MPLAB C32/bin/../lib/gcc/pic32mx/3.4.4/../../../../pic32mx/lib/size\libc.a(stubs.o)
                0x9d01c788                pthread_mutexattr_destroy
                0x9d01c788                _weak_pthread_mutexattr_destroy
 .text._weak_pthread_mutexattr_setname_np
                0x9d01c790        0x8 C:/Program Files/Microchip/MPLAB C32/bin/../lib/gcc/pic32mx/3.4.4/../../../../pic32mx/lib/size\libc.a(stubs.o)
                0x9d01c790                _weak_pthread_mutexattr_setname_np
                0x9d01c790                pthread_mutexattr_setname_np
 .text._weak_pthread_mutexattr_settype_np
                0x9d01c798        0x8 C:/Program Files/Microchip/MPLAB C32/bin/../lib/gcc/pic32mx/3.4.4/../../../../pic32mx/lib/size\libc.a(stubs.o)
                0x9d01c798                _weak_pthread_mutexattr_settype_np
                0x9d01c798                pthread_mutexattr_settype_np
 .text._weak_pthread_sysconf_np
                0x9d01c7a0        0x8 C:/Program Files/Microchip/MPLAB C32/bin/../lib/gcc/pic32mx/3.4.4/../../../../pic32mx/lib/size\libc.a(stubs.o)
                0x9d01c7a0                _weak_pthread_sysconf_np
                0x9d01c7a0                pthread_sysconf_np
 .text._weak_pthread_sigdisable_np
                0x9d01c7a8        0x8 C:/Program Files/Microchip/MPLAB C32/bin/../lib/gcc/pic32mx/3.4.4/../../../../pic32mx/lib/size\libc.a(stubs.o)
                0x9d01c7a8                _weak_pthread_sigdisable_np
                0x9d01c7a8                pthread_sigdisable_np
 .text._weak_pthread_sigrestore_np
                0x9d01c7b0        0x8 C:/Program Files/Microchip/MPLAB C32/bin/../lib/gcc/pic32mx/3.4.4/../../../../pic32mx/lib/size\libc.a(stubs.o)
                0x9d01c7b0                pthread_sigrestore_np
                0x9d01c7b0                _weak_pthread_sigrestore_np
 .text._weak__pthread_cleanup_push
                0x9d01c7b8        0x8 C:/Program Files/Microchip/MPLAB C32/bin/../lib/gcc/pic32mx/3.4.4/../../../../pic32mx/lib/size\libc.a(stubs.o)
                0x9d01c7b8                _weak__pthread_cleanup_push
                0x9d01c7b8                _pthread_cleanup_push
 .text._weak__pthread_cleanup_pop
                0x9d01c7c0        0x8 C:/Program Files/Microchip/MPLAB C32/bin/../lib/gcc/pic32mx/3.4.4/../../../../pic32mx/lib/size\libc.a(stubs.o)
                0x9d01c7c0                _pthread_cleanup_pop
                0x9d01c7c0                _weak__pthread_cleanup_pop
 .text._weak__pthread_cleanup_push_defer
                0x9d01c7c8        0x8 C:/Program Files/Microchip/MPLAB C32/bin/../lib/gcc/pic32mx/3.4.4/../../../../pic32mx/lib/size\libc.a(stubs.o)
                0x9d01c7c8                _weak__pthread_cleanup_push_defer
                0x9d01c7c8                _pthread_cleanup_push_defer
 .text._weak__pthread_cleanup_pop_restore
                0x9d01c7d0        0x8 C:/Program Files/Microchip/MPLAB C32/bin/../lib/gcc/pic32mx/3.4.4/../../../../pic32mx/lib/size\libc.a(stubs.o)
                0x9d01c7d0                _pthread_cleanup_pop_restore
                0x9d01c7d0                _weak__pthread_cleanup_pop_restore
 .text._weak_pthread_once
                0x9d01c7d8       0x2c C:/Program Files/Microchip/MPLAB C32/bin/../lib/gcc/pic32mx/3.4.4/../../../../pic32mx/lib/size\libc.a(stubs.o)
                0x9d01c7d8                _weak_pthread_once
                0x9d01c7d8                pthread_once
                0x9d01c7d8                _pthread_once
 .text._weak_pthread_key_create
                0x9d01c804        0x8 C:/Program Files/Microchip/MPLAB C32/bin/../lib/gcc/pic32mx/3.4.4/../../../../pic32mx/lib/size\libc.a(stubs.o)
                0x9d01c804                pthread_key_create
                0x9d01c804                _weak_pthread_key_create
 .text._weak_pthread_setspecific
                0x9d01c80c        0x8 C:/Program Files/Microchip/MPLAB C32/bin/../lib/gcc/pic32mx/3.4.4/../../../../pic32mx/lib/size\libc.a(stubs.o)
                0x9d01c80c                _weak_pthread_setspecific
                0x9d01c80c                pthread_setspecific
 .text._weak_pthread_getspecific
                0x9d01c814        0x8 C:/Program Files/Microchip/MPLAB C32/bin/../lib/gcc/pic32mx/3.4.4/../../../../pic32mx/lib/size\libc.a(stubs.o)
                0x9d01c814                pthread_getspecific
                0x9d01c814                _weak_pthread_getspecific
 .text._weak__libc_private_storage
                0x9d01c81c        0x8 C:/Program Files/Microchip/MPLAB C32/bin/../lib/gcc/pic32mx/3.4.4/../../../../pic32mx/lib/size\libc.a(stubs.o)
                0x9d01c81c                _libc_private_storage
                0x9d01c81c                _weak__libc_private_storage
 .text._bootstrap_exception_handler
                0x9d01c824        0x8 C:/Program Files/Microchip/MPLAB C32/bin/../lib/gcc/pic32mx/3.4.4/../../../../pic32mx/lib/size\libc.a(default-bootstrap-exception-handler.o)
                0x9d01c824                _bootstrap_exception_handler
 .text._on_reset
                0x9d01c82c        0x8 C:/Program Files/Microchip/MPLAB C32/bin/../lib/gcc/pic32mx/3.4.4/../../../../pic32mx/lib/size\libc.a(default-on-reset.o)
                0x9d01c82c                _on_reset
 .text._on_bootstrap
                0x9d01c834        0x8 C:/Program Files/Microchip/MPLAB C32/bin/../lib/gcc/pic32mx/3.4.4/../../../../pic32mx/lib/size\libc.a(default-on-bootstrap.o)
                0x9d01c834                _on_bootstrap
 .text          0x9d01c83c       0x18 C:/Program Files/Microchip/MPLAB C32/bin/../lib/gcc/pic32mx/3.4.4/../../../../pic32mx/lib/size\libc.a(default-nmi-handler.o)
                0x9d01c83c                _nmi_handler
 .text._mon_getc
                0x9d01c854        0x8 C:/Program Files/Microchip/MPLAB C32/bin/../lib/gcc/pic32mx/3.4.4/../../../../pic32mx/lib/size\libc.a(_mon_getc.o)
                0x9d01c854                _mon_getc
 .text._mon_write
                0x9d01c85c       0x4c C:/Program Files/Microchip/MPLAB C32/bin/../lib/gcc/pic32mx/3.4.4/../../../../pic32mx/lib/size\libc.a(_mon_write.o)
                0x9d01c85c                _mon_write
 .text._exit    0x9d01c8a8        0x8 C:/Program Files/Microchip/MPLAB C32/bin/../lib/gcc/pic32mx/3.4.4/../../../../pic32mx/lib/size\libc.a(_exit.o)
                0x9d01c8a8                _exit
 .text._mon_putc
                0x9d01c8b0       0x28 C:/Program Files/Microchip/MPLAB C32/bin/../lib/gcc/pic32mx/3.4.4/../../../../pic32mx/lib/size\libc.a(_mon_putc.o)
                0x9d01c8b0                _mon_putc
 .text.INTDisableInterrupts
                0x9d01c8d8        0x8 C:/Program Files/Microchip/MPLAB C32/bin/../lib/gcc/pic32mx/3.4.4/../../../../pic32mx/lib/size\libmchp_peripheral.a(int_disable_interrupts_lib.o)
                0x9d01c8d8                INTDisableInterrupts
 .text.INTEnableSystemMultiVectoredInt
                0x9d01c8e0       0x34 C:/Program Files/Microchip/MPLAB C32/bin/../lib/gcc/pic32mx/3.4.4/../../../../pic32mx/lib/size\libmchp_peripheral.a(int_enable_mv_int_lib.o)
                0x9d01c8e0                INTEnableSystemMultiVectoredInt
 .text.INTRestoreInterrupts
                0x9d01c914       0x1c C:/Program Files/Microchip/MPLAB C32/bin/../lib/gcc/pic32mx/3.4.4/../../../../pic32mx/lib/size\libmchp_peripheral.a(int_restore_interrupts_lib.o)
                0x9d01c914                INTRestoreInterrupts
 .text.SoftReset
                0x9d01c930       0x78 C:/Program Files/Microchip/MPLAB C32/bin/../lib/gcc/pic32mx/3.4.4/../../../../pic32mx/lib/size\libmchp_peripheral.a(soft_reset_lib.o)
                0x9d01c930                SoftReset
 .text.CheKseg0CacheOff
                0x9d01c9a8       0x18 C:/Program Files/Microchip/MPLAB C32/bin/../lib/gcc/pic32mx/3.4.4/../../../../pic32mx/lib/size\libmchp_peripheral.a(pcache.o)
                0x9d01c9a8                CheKseg0CacheOff
 .text.CheKseg0CacheOn
                0x9d01c9c0       0x18 C:/Program Files/Microchip/MPLAB C32/bin/../lib/gcc/pic32mx/3.4.4/../../../../pic32mx/lib/size\libmchp_peripheral.a(pcache.o)
                0x9d01c9c0                CheKseg0CacheOn
 .text.INTEnableInterrupts
                0x9d01c9d8        0x8 C:/Program Files/Microchip/MPLAB C32/bin/../lib/gcc/pic32mx/3.4.4/../../../../pic32mx/lib/size\libmchp_peripheral.a(int_enable_interrupts_lib.o)
                0x9d01c9d8                INTEnableInterrupts
 *(.text.*personality*)
 *(.gnu.warning)
 *(.mips16.fn.*)
 *(.mips16.call.*)
                0x9d01c9e0                _text_end = .

.rodata         0x9d01c9e0      0xf1c
 *(.rodata .rodata.* .gnu.linkonce.r.*)
 .rodata        0x9d01c9e0       0x38 Objects - TCPIP Demo App-C32\MainDemo.o
 .rodata        0x9d01ca18       0xec Objects - TCPIP Demo App-C32\CustomHTTPApp.o
 .rodata        0x9d01cb04       0x34 ..\Microchip\TCPIP Stack\Objects - TCPIP Demo App-C32\DHCP.o
 .rodata        0x9d01cb38       0x20 ..\Microchip\TCPIP Stack\Objects - TCPIP Demo App-C32\DNS.o
 .rodata        0x9d01cb58      0x21c ..\Microchip\TCPIP Stack\Objects - TCPIP Demo App-C32\DynDNS.o
 .rodata        0x9d01cd74      0x140 ..\Microchip\TCPIP Stack\Objects - TCPIP Demo App-C32\Hashes.o
 .rodata        0x9d01ceb4      0x46c ..\Microchip\TCPIP Stack\Objects - TCPIP Demo App-C32\HTTP2.o
 .rodata        0x9d01d320        0x8 ..\Microchip\TCPIP Stack\Objects - TCPIP Demo App-C32\MPFS2.o
 .rodata        0x9d01d328      0x1e0 ..\Microchip\TCPIP Stack\Objects - TCPIP Demo App-C32\SMTP.o
 .rodata        0x9d01d508       0xa8 ..\Microchip\TCPIP Stack\Objects - TCPIP Demo App-C32\TCP.o
                0x9d01d508                TCPSocketInitializer
 .rodata        0x9d01d5b0       0x50 Objects - TCPIP Demo App-C32\SMTPDemo.o
 .rodata        0x9d01d600      0x1e4 Objects - TCPIP Demo App-C32\MPFSImg2-C32.o
                0x9d01d600                MPFS_Start
 .rodata        0x9d01d7e4       0x14 C:/Program Files/Microchip/MPLAB C32/bin/../lib/gcc/pic32mx/3.4.4/../../../../pic32mx/lib/size\libc.a(_iobdata.o)
                0x9d01d7e4                _io_funcs
 .rodata        0x9d01d7f8      0x104 C:/Program Files/Microchip/MPLAB C32/bin/../lib/gcc/pic32mx/3.4.4/../../../../pic32mx/lib/size\libc.a(ctype.o)
                0x9d01d7f8                _ctype
 *(.rodata1)
                0x9d01d8fc                . = ALIGN (0x4)

.sdata2         0x9d01d8fc        0x0
 *(.sdata2 .sdata2.* .gnu.linkonce.s2.*)
                0x9d01d8fc                . = ALIGN (0x4)

.sbss2          0x9d01d8fc        0x0
 *(.sbss2 .sbss2.* .gnu.linkonce.sb2.*)
                0x9d01d8fc                . = ALIGN (0x4)

.eh_frame_hdr
 *(.eh_frame_hdr)

.eh_frame       0x9d01d8fc       0x20
 *(.eh_frame)
 .eh_frame      0x9d01d8fc       0x20 C:/Program Files/Microchip/MPLAB C32/bin/../lib/gcc/pic32mx/3.4.4/size\libgcc.a(_udivdi3.o)

.dbg_data       0xa0000000        0x0
                0xa0000000                . = (. + DEFINED (_DEBUGGER)?0x200:0x0)

.data           0xa0000000      0x23c load address 0x9d01d91c
                0xa0000000                _data_begin = .
 *(.data .data.* .gnu.linkonce.d.*)
 .data          0xa0000000       0x40 ..\Microchip\TCPIP Stack\Objects - TCPIP Demo App-C32\DynDNS.o
                0xa0000034                ddnsServiceHosts
 .data          0xa0000040       0x90 ..\Microchip\TCPIP Stack\Objects - TCPIP Demo App-C32\HTTP2.o
 .data          0xa00000d0       0x48 Objects - TCPIP Demo App-C32\SMTPDemo.o
 .data          0xa0000118       0x20 C:/Program Files/Microchip/MPLAB C32/bin/../lib/gcc/pic32mx/3.4.4/../../../../pic32mx/lib/size\libc.a(exit.o)
                0xa0000118                __exfun_mx
 .data          0xa0000138       0x30 C:/Program Files/Microchip/MPLAB C32/bin/../lib/gcc/pic32mx/3.4.4/../../../../pic32mx/lib/size\libc.a(rand.o)
 .data          0xa0000168       0xd4 C:/Program Files/Microchip/MPLAB C32/bin/../lib/gcc/pic32mx/3.4.4/../../../../pic32mx/lib/size\libc.a(_iobdata.o)
 *(.gnu.linkonce.d.*personality*)
 *(.data1)
                0x9d01d91c                _data_image_begin = LOADADDR (.data)

.eh_frame
 *(.eh_frame)
                0xa0008230                _gp = (ALIGN (0x10) + 0x7ff0)

.got
 *(.got.plt)
 *(.got)

.sdata          0xa000023c       0x28 load address 0x9d01db58
                0xa000023c                _sdata_begin = .
 *(.sdata .sdata.* .gnu.linkonce.s.*)
 .sdata         0xa000023c        0x8 Objects - TCPIP Demo App-C32\MainDemo.o
                0xa000023c                myDHCPBindCount
                0xa0000240                __C30_UART
 .sdata         0xa0000244        0x8 ..\Microchip\TCPIP Stack\Objects - TCPIP Demo App-C32\DHCP.o
                0xa0000244                smDHCPState
 .sdata         0xa000024c        0x4 ..\Microchip\TCPIP Stack\Objects - TCPIP Demo App-C32\DHCPs.o
                0xa000024c                bDHCPServerEnabled
 .sdata         0xa0000250        0x8 ..\Microchip\TCPIP Stack\Objects - TCPIP Demo App-C32\DNS.o
 .sdata         0xa0000258        0x1 ..\Microchip\TCPIP Stack\Objects - TCPIP Demo App-C32\DynDNS.o
 .sdata         0xa0000259        0x1 ..\Microchip\TCPIP Stack\Objects - TCPIP Demo App-C32\SMTP.o
 .sdata         0xa000025a        0x2 ..\Microchip\TCPIP Stack\Objects - TCPIP Demo App-C32\TCP.o
 .sdata         0xa000025c        0x2 ..\Microchip\TCPIP Stack\Objects - TCPIP Demo App-C32\UDP.o
 *fill*         0xa000025e        0x2 00
 .sdata         0xa0000260        0x4 C:/Program Files/Microchip/MPLAB C32/bin/../lib/gcc/pic32mx/3.4.4/../../../../pic32mx/lib/size\libc.a(_iobdata.o)
                0xa0000260                _libc_data
                0xa0000264                _sdata_end = .

.lit8
 *(.lit8)

.lit4
 *(.lit4)
                0xa0000264                . = ALIGN (0x4)
                0xa0000264                _data_end = .
                0xa0000264                _bss_begin = .

.sbss           0xa0000264      0x110
                0xa0000264                _sbss_begin = .
 *(.dynsbss)
 *(.sbss .sbss.* .gnu.linkonce.sb.*)
 .sbss          0xa0000264        0x4 Objects - TCPIP Demo App-C32\MainDemo.o
 .sbss          0xa0000268        0x4 ..\Microchip\TCPIP Stack\Objects - TCPIP Demo App-C32\ARP.o
 .sbss          0xa000026c       0x28 ..\Microchip\TCPIP Stack\Objects - TCPIP Demo App-C32\DHCP.o
                0xa000026d                DHCPBindCount
                0xa000026c                DHCPFlags
 .sbss          0xa0000294        0xc ..\Microchip\TCPIP Stack\Objects - TCPIP Demo App-C32\DHCPs.o
 .sbss          0xa00002a0       0x18 ..\Microchip\TCPIP Stack\Objects - TCPIP Demo App-C32\DNS.o
 .sbss          0xa00002b8       0x24 ..\Microchip\TCPIP Stack\Objects - TCPIP Demo App-C32\DynDNS.o
 .sbss          0xa00002dc       0x10 ..\Microchip\TCPIP Stack\Objects - TCPIP Demo App-C32\ENC28J60.o
 .sbss          0xa00002ec        0x4 ..\Microchip\TCPIP Stack\Objects - TCPIP Demo App-C32\IP.o
 .sbss          0xa00002f0        0x8 ..\Microchip\TCPIP Stack\Objects - TCPIP Demo App-C32\MPFS2.o
 .sbss          0xa00002f8        0x8 ..\Microchip\TCPIP Stack\Objects - TCPIP Demo App-C32\NBNS.o
 .sbss          0xa0000300       0x38 ..\Microchip\TCPIP Stack\Objects - TCPIP Demo App-C32\SMTP.o
 .sbss          0xa0000338        0x4 ..\Microchip\TCPIP Stack\Objects - TCPIP Demo App-C32\StackTsk.o
 .sbss          0xa000033c        0x2 ..\Microchip\TCPIP Stack\Objects - TCPIP Demo App-C32\TCP.o
 *fill*         0xa000033e        0x2 00
 .sbss          0xa0000340        0xc ..\Microchip\TCPIP Stack\Objects - TCPIP Demo App-C32\Tick.o
 .sbss          0xa000034c        0xc ..\Microchip\TCPIP Stack\Objects - TCPIP Demo App-C32\UDP.o
 .sbss          0xa0000358        0x8 Objects - TCPIP Demo App-C32\SMTPDemo.o
 .sbss          0xa0000360        0x4 C:/Program Files/Microchip/MPLAB C32/bin/../lib/gcc/pic32mx/3.4.4/../../../../pic32mx/lib/size\libc.a(errno.o)
                0xa0000360                errno
 *(.scommon)
 .scommon       0xa0000364        0x8 Objects - TCPIP Demo App-C32\MainDemo.o
                0xa0000364                AN0String
 .scommon       0xa000036c        0x1 ..\Microchip\TCPIP Stack\Objects - TCPIP Demo App-C32\HTTP2.o
                0xa000036c                curHTTPID
 *fill*         0xa000036d        0x1 00
 .scommon       0xa000036e        0x6 ..\Microchip\TCPIP Stack\Objects - TCPIP Demo App-C32\UDP.o
                0xa000036e                UDPTxCount
                0xa0000370                activeUDPSocket
                0xa0000372                UDPRxCount
                0xa0000374                _sbss_end = .

.bss            0xa0000374      0x6f8
 *(.dynbss)
 *(.bss .bss.* .gnu.linkonce.b.*)
 .bss           0xa0000374       0x18 ..\Microchip\TCPIP Stack\Objects - TCPIP Demo App-C32\ARP.o
 .bss           0xa000038c        0xc ..\Microchip\TCPIP Stack\Objects - TCPIP Demo App-C32\DNS.o
 .bss           0xa0000398       0x10 ..\Microchip\TCPIP Stack\Objects - TCPIP Demo App-C32\DynDNS.o
 .bss           0xa00003a8       0x78 ..\Microchip\TCPIP Stack\Objects - TCPIP Demo App-C32\MPFS2.o
 .bss           0xa0000420      0x224 ..\Microchip\TCPIP Stack\Objects - TCPIP Demo App-C32\TCP.o
 .bss           0xa0000644       0x88 C:/Program Files/Microchip/MPLAB C32/bin/../lib/gcc/pic32mx/3.4.4/../../../../pic32mx/lib/size\libc.a(_iobdata.o)
 .bss           0xa00006cc       0x80 C:/Program Files/Microchip/MPLAB C32/bin/../lib/gcc/pic32mx/3.4.4/../../../../pic32mx/lib/size\libc.a(_iobfuncs.o)
 .bss           0xa000074c        0x4 C:/Program Files/Microchip/MPLAB C32/bin/../lib/gcc/pic32mx/3.4.4/../../../../pic32mx/lib/size\libc.a(stubs.o)
                0xa000074c                __isthreaded
 *(COMMON)
 COMMON         0xa0000750       0x33 Objects - TCPIP Demo App-C32\MainDemo.o
                0xa0000750                AppConfig
 *fill*         0xa0000783        0x1 00
 COMMON         0xa0000784      0x102 Objects - TCPIP Demo App-C32\CustomHTTPApp.o
                0xa0000784                bufWeight
                0xa00007b8                bufHeight
                0xa00007ec                bufName
                0xa0000820                bufEye
                0xa0000854                bufGender
 *fill*         0xa0000886        0x2 00
 COMMON         0xa0000888       0x20 ..\Microchip\TCPIP Stack\Objects - TCPIP Demo App-C32\DynDNS.o
                0xa0000888                DDNSClient
 COMMON         0xa00008a8       0x40 ..\Microchip\TCPIP Stack\Objects - TCPIP Demo App-C32\Hashes.o
                0xa00008a8                lastBlock
 COMMON         0xa00008e8       0x9c ..\Microchip\TCPIP Stack\Objects - TCPIP Demo App-C32\HTTP2.o
                0xa00008e8                curHTTP
                0xa0000974                httpStubs
 COMMON         0xa0000984       0x21 ..\Microchip\TCPIP Stack\Objects - TCPIP Demo App-C32\LCDBlocking.o
                0xa0000984                LCDText
 *fill*         0xa00009a5        0x3 00
 COMMON         0xa00009a8       0x2c ..\Microchip\TCPIP Stack\Objects - TCPIP Demo App-C32\SMTP.o
                0xa00009a8                SMTPClient
 COMMON         0xa00009d4        0xa ..\Microchip\TCPIP Stack\Objects - TCPIP Demo App-C32\StackTsk.o
                0xa00009d4                remoteNode
 *fill*         0xa00009de        0x2 00
 COMMON         0xa00009e0       0x8c ..\Microchip\TCPIP Stack\Objects - TCPIP Demo App-C32\UDP.o
                0xa00009e0                UDPSocketInfo
                0xa0000a6c                . = ALIGN (0x4)
                0xa0000a6c                . = ALIGN (0x4)
                0xa0000a6c                _end = .
                0xa0000a6c                _bss_end = .

.heap           0xa0000a6c        0x0
                0xa0000a6c                _heap = .
                0xa0000a6c                . = (. + _min_heap_size)

.stack          0xa0000a6c      0x400
                0xa0000e6c                . = (. + _min_stack_size)
 *fill*         0xa0000a6c      0x400 00

.ramfunc        0xa0001000        0x0 load address 0x9d01db80
                0xa0001000                _ramfunc_begin = .
 *(.ramfunc .ramfunc.*)
                0xa0001000                . = ALIGN (0x4)
                0xa0001000                _ramfunc_end = .
                0x9d01db80                _ramfunc_image_begin = LOADADDR (.ramfunc)
                0x00000000                _ramfunc_length = SIZEOF (.ramfunc)
                0x00001000                _bmxdkpba_address = (_ramfunc_begin - 0xa0000000)
                0x00008000                _bmxdudba_address = 0x8000
                0x00008000                _bmxdupba_address = 0x8000
                0xa0008000                _stack = (_ramfunc_length > 0x0)?(_ramfunc_begin - 0x4):0xa0008000
                0x00000001                ASSERT (((_min_stack_size + _min_heap_size) <= (_stack - _heap)), Not enough space to allocate both stack and heap.  Reduce heap and/or stack size.)

.pdr            0x00000000     0x2260
 *(.pdr)
 .pdr           0x00000000       0xa0 C:/Program Files/Microchip/MPLAB C32/bin/../lib/gcc/pic32mx/3.4.4/../../../../pic32mx/lib/size/crt0.o
 .pdr           0x000000a0       0xc0 Objects - TCPIP Demo App-C32\MainDemo.o
 .pdr           0x00000160       0x80 Objects - TCPIP Demo App-C32\CustomHTTPApp.o
 .pdr           0x000001e0       0xc0 ..\Microchip\TCPIP Stack\Objects - TCPIP Demo App-C32\ARP.o
 .pdr           0x000002a0       0x40 ..\Microchip\TCPIP Stack\Objects - TCPIP Demo App-C32\Delay.o
 .pdr           0x000002e0       0xc0 ..\Microchip\TCPIP Stack\Objects - TCPIP Demo App-C32\DHCP.o
 .pdr           0x000003a0       0x60 ..\Microchip\TCPIP Stack\Objects - TCPIP Demo App-C32\DHCPs.o
 .pdr           0x00000400       0xc0 ..\Microchip\TCPIP Stack\Objects - TCPIP Demo App-C32\DNS.o
 .pdr           0x000004c0       0xc0 ..\Microchip\TCPIP Stack\Objects - TCPIP Demo App-C32\DynDNS.o
 .pdr           0x00000580      0x400 ..\Microchip\TCPIP Stack\Objects - TCPIP Demo App-C32\ENC28J60.o
 .pdr           0x00000980       0xa0 ..\Microchip\TCPIP Stack\Objects - TCPIP Demo App-C32\Hashes.o
 .pdr           0x00000a20      0x1e0 ..\Microchip\TCPIP Stack\Objects - TCPIP Demo App-C32\Helpers.o
 .pdr           0x00000c00      0x220 ..\Microchip\TCPIP Stack\Objects - TCPIP Demo App-C32\HTTP2.o
 .pdr           0x00000e20       0x20 ..\Microchip\TCPIP Stack\Objects - TCPIP Demo App-C32\ICMP.o
 .pdr           0x00000e40       0x80 ..\Microchip\TCPIP Stack\Objects - TCPIP Demo App-C32\IP.o
 .pdr           0x00000ec0       0x80 ..\Microchip\TCPIP Stack\Objects - TCPIP Demo App-C32\LCDBlocking.o
 .pdr           0x00000f40      0x280 ..\Microchip\TCPIP Stack\Objects - TCPIP Demo App-C32\MPFS2.o
 .pdr           0x000011c0       0x60 ..\Microchip\TCPIP Stack\Objects - TCPIP Demo App-C32\NBNS.o
 .pdr           0x00001220      0x1a0 ..\Microchip\TCPIP Stack\Objects - TCPIP Demo App-C32\SMTP.o
 .pdr           0x000013c0       0x60 ..\Microchip\TCPIP Stack\Objects - TCPIP Demo App-C32\StackTsk.o
 .pdr           0x00001420      0x3a0 ..\Microchip\TCPIP Stack\Objects - TCPIP Demo App-C32\TCP.o
 .pdr           0x000017c0      0x100 ..\Microchip\TCPIP Stack\Objects - TCPIP Demo App-C32\Tick.o
 .pdr           0x000018c0      0x220 ..\Microchip\TCPIP Stack\Objects - TCPIP Demo App-C32\UDP.o
 .pdr           0x00001ae0       0x20 Objects - TCPIP Demo App-C32\SMTPDemo.o
 .pdr           0x00001b00       0x20 C:/Program Files/Microchip/MPLAB C32/bin/../lib/gcc/pic32mx/3.4.4/size\libgcc.a(_udivdi3.o)
 .pdr           0x00001b20       0x20 C:/Program Files/Microchip/MPLAB C32/bin/../lib/gcc/pic32mx/3.4.4/../../../../pic32mx/lib/size\libc.a(memcmp.o)
 .pdr           0x00001b40       0x20 C:/Program Files/Microchip/MPLAB C32/bin/../lib/gcc/pic32mx/3.4.4/../../../../pic32mx/lib/size\libc.a(memcpy.o)
 .pdr           0x00001b60       0x20 C:/Program Files/Microchip/MPLAB C32/bin/../lib/gcc/pic32mx/3.4.4/../../../../pic32mx/lib/size\libc.a(memset.o)
 .pdr           0x00001b80       0x20 C:/Program Files/Microchip/MPLAB C32/bin/../lib/gcc/pic32mx/3.4.4/../../../../pic32mx/lib/size\libc.a(strcmp.o)
 .pdr           0x00001ba0       0x20 C:/Program Files/Microchip/MPLAB C32/bin/../lib/gcc/pic32mx/3.4.4/../../../../pic32mx/lib/size\libc.a(strcpy.o)
 .pdr           0x00001bc0       0x20 C:/Program Files/Microchip/MPLAB C32/bin/../lib/gcc/pic32mx/3.4.4/../../../../pic32mx/lib/size\libc.a(strlen.o)
 .pdr           0x00001be0       0x20 C:/Program Files/Microchip/MPLAB C32/bin/../lib/gcc/pic32mx/3.4.4/../../../../pic32mx/lib/size\libc.a(general-exception.o)
 .pdr           0x00001c00       0x20 C:/Program Files/Microchip/MPLAB C32/bin/../lib/gcc/pic32mx/3.4.4/../../../../pic32mx/lib/size\libc.a(strchr.o)
 .pdr           0x00001c20       0x20 C:/Program Files/Microchip/MPLAB C32/bin/../lib/gcc/pic32mx/3.4.4/../../../../pic32mx/lib/size\libc.a(strstr.o)
 .pdr           0x00001c40       0x20 C:/Program Files/Microchip/MPLAB C32/bin/../lib/gcc/pic32mx/3.4.4/../../../../pic32mx/lib/size\libc.a(exit.o)
 .pdr           0x00001c60       0x60 C:/Program Files/Microchip/MPLAB C32/bin/../lib/gcc/pic32mx/3.4.4/../../../../pic32mx/lib/size\libc.a(rand.o)
 .pdr           0x00001cc0       0x20 C:/Program Files/Microchip/MPLAB C32/bin/../lib/gcc/pic32mx/3.4.4/../../../../pic32mx/lib/size\libc.a(atol.o)
 .pdr           0x00001ce0       0x20 C:/Program Files/Microchip/MPLAB C32/bin/../lib/gcc/pic32mx/3.4.4/../../../../pic32mx/lib/size\libc.a(atoi.o)
 .pdr           0x00001d00       0x20 C:/Program Files/Microchip/MPLAB C32/bin/../lib/gcc/pic32mx/3.4.4/../../../../pic32mx/lib/size\libc.a(strtol.o)
 .pdr           0x00001d20       0xa0 C:/Program Files/Microchip/MPLAB C32/bin/../lib/gcc/pic32mx/3.4.4/../../../../pic32mx/lib/size\libc.a(_iobfuncs.o)
 .pdr           0x00001dc0      0x2c0 C:/Program Files/Microchip/MPLAB C32/bin/../lib/gcc/pic32mx/3.4.4/../../../../pic32mx/lib/size\libc.a(stubs.o)
 .pdr           0x00002080       0x20 C:/Program Files/Microchip/MPLAB C32/bin/../lib/gcc/pic32mx/3.4.4/../../../../pic32mx/lib/size\libc.a(default-bootstrap-exception-handler.o)
 .pdr           0x000020a0       0x20 C:/Program Files/Microchip/MPLAB C32/bin/../lib/gcc/pic32mx/3.4.4/../../../../pic32mx/lib/size\libc.a(default-on-reset.o)
 .pdr           0x000020c0       0x20 C:/Program Files/Microchip/MPLAB C32/bin/../lib/gcc/pic32mx/3.4.4/../../../../pic32mx/lib/size\libc.a(default-on-bootstrap.o)
 .pdr           0x000020e0       0x20 C:/Program Files/Microchip/MPLAB C32/bin/../lib/gcc/pic32mx/3.4.4/../../../../pic32mx/lib/size\libc.a(default-nmi-handler.o)
 .pdr           0x00002100       0x20 C:/Program Files/Microchip/MPLAB C32/bin/../lib/gcc/pic32mx/3.4.4/../../../../pic32mx/lib/size\libc.a(_mon_getc.o)
 .pdr           0x00002120       0x20 C:/Program Files/Microchip/MPLAB C32/bin/../lib/gcc/pic32mx/3.4.4/../../../../pic32mx/lib/size\libc.a(_mon_write.o)
 .pdr           0x00002140       0x20 C:/Program Files/Microchip/MPLAB C32/bin/../lib/gcc/pic32mx/3.4.4/../../../../pic32mx/lib/size\libc.a(_exit.o)
 .pdr           0x00002160       0x20 C:/Program Files/Microchip/MPLAB C32/bin/../lib/gcc/pic32mx/3.4.4/../../../../pic32mx/lib/size\libc.a(_mon_putc.o)
 .pdr           0x00002180       0x20 C:/Program Files/Microchip/MPLAB C32/bin/../lib/gcc/pic32mx/3.4.4/../../../../pic32mx/lib/size\libmchp_peripheral.a(int_disable_interrupts_lib.o)
 .pdr           0x000021a0       0x20 C:/Program Files/Microchip/MPLAB C32/bin/../lib/gcc/pic32mx/3.4.4/../../../../pic32mx/lib/size\libmchp_peripheral.a(int_enable_mv_int_lib.o)
 .pdr           0x000021c0       0x20 C:/Program Files/Microchip/MPLAB C32/bin/../lib/gcc/pic32mx/3.4.4/../../../../pic32mx/lib/size\libmchp_peripheral.a(int_restore_interrupts_lib.o)
 .pdr           0x000021e0       0x20 C:/Program Files/Microchip/MPLAB C32/bin/../lib/gcc/pic32mx/3.4.4/../../../../pic32mx/lib/size\libmchp_peripheral.a(soft_reset_lib.o)
 .pdr           0x00002200       0x40 C:/Program Files/Microchip/MPLAB C32/bin/../lib/gcc/pic32mx/3.4.4/../../../../pic32mx/lib/size\libmchp_peripheral.a(pcache.o)
 .pdr           0x00002240       0x20 C:/Program Files/Microchip/MPLAB C32/bin/../lib/gcc/pic32mx/3.4.4/../../../../pic32mx/lib/size\libmchp_peripheral.a(int_enable_interrupts_lib.o)

.reginfo        0x00000000       0x18
 *(.reginfo)
 .reginfo       0x00000000       0x18 C:/Program Files/Microchip/MPLAB C32/bin/../lib/gcc/pic32mx/3.4.4/../../../../pic32mx/lib/size/crt0.o

.stab
 *(.stab)

.stabstr
 *(.stabstr)

.stab.excl
 *(.stab.excl)

.stab.exclstr
 *(.stab.exclstr)

.stab.index
 *(.stab.index)

.stab.indexstr
 *(.stab.indexstr)

.comment        0x00000000     0x1e57
 *(.comment)
 .comment       0x00000000       0x4d Objects - TCPIP Demo App-C32\MainDemo.o
 .comment       0x0000004d       0x4d Objects - TCPIP Demo App-C32\CustomHTTPApp.o
 .comment       0x0000009a       0x4d ..\Microchip\TCPIP Stack\Objects - TCPIP Demo App-C32\UDPPerformanceTest.o
 .comment       0x000000e7       0x4d ..\Microchip\TCPIP Stack\Objects - TCPIP Demo App-C32\Announce.o
 .comment       0x00000134       0x4d ..\Microchip\TCPIP Stack\Objects - TCPIP Demo App-C32\ARP.o
 .comment       0x00000181       0x4d ..\Microchip\TCPIP Stack\Objects - TCPIP Demo App-C32\Delay.o
 .comment       0x000001ce       0x4d ..\Microchip\TCPIP Stack\Objects - TCPIP Demo App-C32\DHCP.o
 .comment       0x0000021b       0x4d ..\Microchip\TCPIP Stack\Objects - TCPIP Demo App-C32\DHCPs.o
 .comment       0x00000268       0x4d ..\Microchip\TCPIP Stack\Objects - TCPIP Demo App-C32\DNS.o
 .comment       0x000002b5       0x4d ..\Microchip\TCPIP Stack\Objects - TCPIP Demo App-C32\DynDNS.o
 .comment       0x00000302       0x4d ..\Microchip\TCPIP Stack\Objects - TCPIP Demo App-C32\ENC28J60.o
 .comment       0x0000034f       0x4d ..\Microchip\TCPIP Stack\Objects - TCPIP Demo App-C32\FTP.o
 .comment       0x0000039c       0x4d ..\Microchip\TCPIP Stack\Objects - TCPIP Demo App-C32\Hashes.o
 .comment       0x000003e9       0x4d ..\Microchip\TCPIP Stack\Objects - TCPIP Demo App-C32\Helpers.o
 .comment       0x00000436       0x4d ..\Microchip\TCPIP Stack\Objects - TCPIP Demo App-C32\HTTP2.o
 .comment       0x00000483       0x4d ..\Microchip\TCPIP Stack\Objects - TCPIP Demo App-C32\HTTP.o
 .comment       0x000004d0       0x4d ..\Microchip\TCPIP Stack\Objects - TCPIP Demo App-C32\ICMP.o
 .comment       0x0000051d       0x4d ..\Microchip\TCPIP Stack\Objects - TCPIP Demo App-C32\IP.o
 .comment       0x0000056a       0x4d ..\Microchip\TCPIP Stack\Objects - TCPIP Demo App-C32\LCDBlocking.o
 .comment       0x000005b7       0x4d ..\Microchip\TCPIP Stack\Objects - TCPIP Demo App-C32\MPFS2.o
 .comment       0x00000604       0x4d ..\Microchip\TCPIP Stack\Objects - TCPIP Demo App-C32\MPFS.o
 .comment       0x00000651       0x4d ..\Microchip\TCPIP Stack\Objects - TCPIP Demo App-C32\NBNS.o
 .comment       0x0000069e       0x4d ..\Microchip\TCPIP Stack\Objects - TCPIP Demo App-C32\Reboot.o
 .comment       0x000006eb       0x4d ..\Microchip\TCPIP Stack\Objects - TCPIP Demo App-C32\SMTP.o
 .comment       0x00000738       0x4d ..\Microchip\TCPIP Stack\Objects - TCPIP Demo App-C32\SNMP.o
 .comment       0x00000785       0x4d ..\Microchip\TCPIP Stack\Objects - TCPIP Demo App-C32\SNTP.o
 .comment       0x000007d2       0x4d ..\Microchip\TCPIP Stack\Objects - TCPIP Demo App-C32\SPIEEPROM.o
 .comment       0x0000081f       0x4d ..\Microchip\TCPIP Stack\Objects - TCPIP Demo App-C32\SPIFlash.o
 .comment       0x0000086c       0x4d ..\Microchip\TCPIP Stack\Objects - TCPIP Demo App-C32\SPIRAM.o
 .comment       0x000008b9       0x4d ..\Microchip\TCPIP Stack\Objects - TCPIP Demo App-C32\StackTsk.o
 .comment       0x00000906       0x4d ..\Microchip\TCPIP Stack\Objects - TCPIP Demo App-C32\TCP.o
 .comment       0x00000953       0x4d ..\Microchip\TCPIP Stack\Objects - TCPIP Demo App-C32\TCPPerformanceTest.o
 .comment       0x000009a0       0x4d ..\Microchip\TCPIP Stack\Objects - TCPIP Demo App-C32\Telnet.o
 .comment       0x000009ed       0x4d ..\Microchip\TCPIP Stack\Objects - TCPIP Demo App-C32\TFTPc.o
 .comment       0x00000a3a       0x4d ..\Microchip\TCPIP Stack\Objects - TCPIP Demo App-C32\Tick.o
 .comment       0x00000a87       0x4d ..\Microchip\TCPIP Stack\Objects - TCPIP Demo App-C32\UART2TCPBridge.o
 .comment       0x00000ad4       0x4d ..\Microchip\TCPIP Stack\Objects - TCPIP Demo App-C32\UART.o
 .comment       0x00000b21       0x4d ..\Microchip\TCPIP Stack\Objects - TCPIP Demo App-C32\UDP.o
 .comment       0x00000b6e       0x4d Objects - TCPIP Demo App-C32\CustomSNMPApp.o
 .comment       0x00000bbb       0x4d Objects - TCPIP Demo App-C32\UARTConfig.o
 .comment       0x00000c08       0x4d Objects - TCPIP Demo App-C32\GenericTCPClient.o
 .comment       0x00000c55       0x4d Objects - TCPIP Demo App-C32\GenericTCPServer.o
 .comment       0x00000ca2       0x4d Objects - TCPIP Demo App-C32\LegacyHTTPApp.o
 .comment       0x00000cef       0x4d Objects - TCPIP Demo App-C32\PingDemo.o
 .comment       0x00000d3c       0x4d Objects - TCPIP Demo App-C32\SMTPDemo.o
 .comment       0x00000d89       0x4d ..\Microchip\TCPIP Stack\Objects - TCPIP Demo App-C32\BerkeleyAPI.o
 .comment       0x00000dd6       0x4d Objects - TCPIP Demo App-C32\BerkeleyUDPClientDemo.o
 .comment       0x00000e23       0x4d Objects - TCPIP Demo App-C32\BerkeleyTCPClientDemo.o
 .comment       0x00000e70       0x4d Objects - TCPIP Demo App-C32\BerkeleyTCPServerDemo.o
 .comment       0x00000ebd       0x4d ..\Microchip\TCPIP Stack\Objects - TCPIP Demo App-C32\ENCX24J600.o
 .comment       0x00000f0a       0x4d ..\Microchip\TCPIP Stack\Objects - TCPIP Demo App-C32\Random.o
 .comment       0x00000f57       0x4d ..\Microchip\TCPIP Stack\Objects - TCPIP Demo App-C32\RSA.o
 .comment       0x00000fa4       0x4d ..\Microchip\TCPIP Stack\Objects - TCPIP Demo App-C32\SSL.o
 .comment       0x00000ff1       0x4d ..\Microchip\TCPIP Stack\Objects - TCPIP Demo App-C32\ARCFOUR.o
 .comment       0x0000103e       0x4d ..\Microchip\TCPIP Stack\Objects - TCPIP Demo App-C32\BigInt.o
 .comment       0x0000108b       0x4d Objects - TCPIP Demo App-C32\CustomSSLCert.o
 .comment       0x000010d8       0x4d Objects - TCPIP Demo App-C32\MPFSImg2-C32.o
 .comment       0x00001125       0x4d C:/Program Files/Microchip/MPLAB C32/bin/../lib/gcc/pic32mx/3.4.4/size\libgcc.a(_udivdi3.o)
 .comment       0x00001172       0x56 C:/Program Files/Microchip/MPLAB C32/bin/../lib/gcc/pic32mx/3.4.4/../../../../pic32mx/lib/size\libc.a(memcmp.o)
 .comment       0x000011c8       0x56 C:/Program Files/Microchip/MPLAB C32/bin/../lib/gcc/pic32mx/3.4.4/../../../../pic32mx/lib/size\libc.a(memset.o)
 .comment       0x0000121e       0x56 C:/Program Files/Microchip/MPLAB C32/bin/../lib/gcc/pic32mx/3.4.4/../../../../pic32mx/lib/size\libc.a(strcmp.o)
 .comment       0x00001274       0x56 C:/Program Files/Microchip/MPLAB C32/bin/../lib/gcc/pic32mx/3.4.4/../../../../pic32mx/lib/size\libc.a(strcpy.o)
 .comment       0x000012ca       0x56 C:/Program Files/Microchip/MPLAB C32/bin/../lib/gcc/pic32mx/3.4.4/../../../../pic32mx/lib/size\libc.a(strlen.o)
 .comment       0x00001320       0x9c C:/Program Files/Microchip/MPLAB C32/bin/../lib/gcc/pic32mx/3.4.4/../../../../pic32mx/lib/size\libc.a(strchr.o)
 .comment       0x000013bc       0x9c C:/Program Files/Microchip/MPLAB C32/bin/../lib/gcc/pic32mx/3.4.4/../../../../pic32mx/lib/size\libc.a(strstr.o)
 .comment       0x00001458       0x9a C:/Program Files/Microchip/MPLAB C32/bin/../lib/gcc/pic32mx/3.4.4/../../../../pic32mx/lib/size\libc.a(exit.o)
 .comment       0x000014f2       0x9a C:/Program Files/Microchip/MPLAB C32/bin/../lib/gcc/pic32mx/3.4.4/../../../../pic32mx/lib/size\libc.a(rand.o)
 .comment       0x0000158c       0x9a C:/Program Files/Microchip/MPLAB C32/bin/../lib/gcc/pic32mx/3.4.4/../../../../pic32mx/lib/size\libc.a(atol.o)
 .comment       0x00001626       0x9a C:/Program Files/Microchip/MPLAB C32/bin/../lib/gcc/pic32mx/3.4.4/../../../../pic32mx/lib/size\libc.a(atoi.o)
 .comment       0x000016c0       0x9c C:/Program Files/Microchip/MPLAB C32/bin/../lib/gcc/pic32mx/3.4.4/../../../../pic32mx/lib/size\libc.a(strtol.o)
 .comment       0x0000175c       0xa0 C:/Program Files/Microchip/MPLAB C32/bin/../lib/gcc/pic32mx/3.4.4/../../../../pic32mx/lib/size\libc.a(_iobdata.o)
 .comment       0x000017fc       0xa1 C:/Program Files/Microchip/MPLAB C32/bin/../lib/gcc/pic32mx/3.4.4/../../../../pic32mx/lib/size\libc.a(_iobfuncs.o)
 .comment       0x0000189d       0x9b C:/Program Files/Microchip/MPLAB C32/bin/../lib/gcc/pic32mx/3.4.4/../../../../pic32mx/lib/size\libc.a(stubs.o)
 .comment       0x00001938       0x4d C:/Program Files/Microchip/MPLAB C32/bin/../lib/gcc/pic32mx/3.4.4/../../../../pic32mx/lib/size\libc.a(default-bootstrap-exception-handler.o)
 .comment       0x00001985       0x4d C:/Program Files/Microchip/MPLAB C32/bin/../lib/gcc/pic32mx/3.4.4/../../../../pic32mx/lib/size\libc.a(default-on-reset.o)
 .comment       0x000019d2       0x4d C:/Program Files/Microchip/MPLAB C32/bin/../lib/gcc/pic32mx/3.4.4/../../../../pic32mx/lib/size\libc.a(default-on-bootstrap.o)
 .comment       0x00001a1f       0x4d C:/Program Files/Microchip/MPLAB C32/bin/../lib/gcc/pic32mx/3.4.4/../../../../pic32mx/lib/size\libc.a(_mon_getc.o)
 .comment       0x00001a6c       0x4d C:/Program Files/Microchip/MPLAB C32/bin/../lib/gcc/pic32mx/3.4.4/../../../../pic32mx/lib/size\libc.a(_mon_write.o)
 .comment       0x00001ab9       0x4d C:/Program Files/Microchip/MPLAB C32/bin/../lib/gcc/pic32mx/3.4.4/../../../../pic32mx/lib/size\libc.a(_exit.o)
 .comment       0x00001b06       0x9b C:/Program Files/Microchip/MPLAB C32/bin/../lib/gcc/pic32mx/3.4.4/../../../../pic32mx/lib/size\libc.a(ctype.o)
 .comment       0x00001ba1       0x9b C:/Program Files/Microchip/MPLAB C32/bin/../lib/gcc/pic32mx/3.4.4/../../../../pic32mx/lib/size\libc.a(errno.o)
 .comment       0x00001c3c       0x4d C:/Program Files/Microchip/MPLAB C32/bin/../lib/gcc/pic32mx/3.4.4/../../../../pic32mx/lib/size\libc.a(_mon_putc.o)
 .comment       0x00001c89       0x4d C:/Program Files/Microchip/MPLAB C32/bin/../lib/gcc/pic32mx/3.4.4/../../../../pic32mx/lib/size\libmchp_peripheral.a(int_disable_interrupts_lib.o)
 .comment       0x00001cd6       0x4d C:/Program Files/Microchip/MPLAB C32/bin/../lib/gcc/pic32mx/3.4.4/../../../../pic32mx/lib/size\libmchp_peripheral.a(int_enable_mv_int_lib.o)
 .comment       0x00001d23       0x4d C:/Program Files/Microchip/MPLAB C32/bin/../lib/gcc/pic32mx/3.4.4/../../../../pic32mx/lib/size\libmchp_peripheral.a(int_restore_interrupts_lib.o)
 .comment       0x00001d70       0x4d C:/Program Files/Microchip/MPLAB C32/bin/../lib/gcc/pic32mx/3.4.4/../../../../pic32mx/lib/size\libmchp_peripheral.a(soft_reset_lib.o)
 .comment       0x00001dbd       0x4d C:/Program Files/Microchip/MPLAB C32/bin/../lib/gcc/pic32mx/3.4.4/../../../../pic32mx/lib/size\libmchp_peripheral.a(pcache.o)
 .comment       0x00001e0a       0x4d C:/Program Files/Microchip/MPLAB C32/bin/../lib/gcc/pic32mx/3.4.4/../../../../pic32mx/lib/size\libmchp_peripheral.a(int_enable_interrupts_lib.o)

.debug
 *(.debug)

.line
 *(.line)

.debug_srcinfo
 *(.debug_srcinfo)

.debug_sfnames
 *(.debug_sfnames)

.debug_aranges  0x00000000      0x730
 *(.debug_aranges)
 .debug_aranges
                0x00000000       0x20 Objects - TCPIP Demo App-C32\MainDemo.o
 .debug_aranges
                0x00000020       0x20 Objects - TCPIP Demo App-C32\CustomHTTPApp.o
 .debug_aranges
                0x00000040       0x20 ..\Microchip\TCPIP Stack\Objects - TCPIP Demo App-C32\ARP.o
 .debug_aranges
                0x00000060       0x20 ..\Microchip\TCPIP Stack\Objects - TCPIP Demo App-C32\Delay.o
 .debug_aranges
                0x00000080       0x20 ..\Microchip\TCPIP Stack\Objects - TCPIP Demo App-C32\DHCP.o
 .debug_aranges
                0x000000a0       0x20 ..\Microchip\TCPIP Stack\Objects - TCPIP Demo App-C32\DHCPs.o
 .debug_aranges
                0x000000c0       0x20 ..\Microchip\TCPIP Stack\Objects - TCPIP Demo App-C32\DNS.o
 .debug_aranges
                0x000000e0       0x20 ..\Microchip\TCPIP Stack\Objects - TCPIP Demo App-C32\DynDNS.o
 .debug_aranges
                0x00000100       0x20 ..\Microchip\TCPIP Stack\Objects - TCPIP Demo App-C32\ENC28J60.o
 .debug_aranges
                0x00000120       0x20 ..\Microchip\TCPIP Stack\Objects - TCPIP Demo App-C32\Hashes.o
 .debug_aranges
                0x00000140       0x20 ..\Microchip\TCPIP Stack\Objects - TCPIP Demo App-C32\Helpers.o
 .debug_aranges
                0x00000160       0x20 ..\Microchip\TCPIP Stack\Objects - TCPIP Demo App-C32\HTTP2.o
 .debug_aranges
                0x00000180       0x20 ..\Microchip\TCPIP Stack\Objects - TCPIP Demo App-C32\ICMP.o
 .debug_aranges
                0x000001a0       0x20 ..\Microchip\TCPIP Stack\Objects - TCPIP Demo App-C32\IP.o
 .debug_aranges
                0x000001c0       0x20 ..\Microchip\TCPIP Stack\Objects - TCPIP Demo App-C32\LCDBlocking.o
 .debug_aranges
                0x000001e0       0x20 ..\Microchip\TCPIP Stack\Objects - TCPIP Demo App-C32\MPFS2.o
 .debug_aranges
                0x00000200       0x20 ..\Microchip\TCPIP Stack\Objects - TCPIP Demo App-C32\NBNS.o
 .debug_aranges
                0x00000220       0x20 ..\Microchip\TCPIP Stack\Objects - TCPIP Demo App-C32\SMTP.o
 .debug_aranges
                0x00000240       0x20 ..\Microchip\TCPIP Stack\Objects - TCPIP Demo App-C32\StackTsk.o
 .debug_aranges
                0x00000260       0x20 ..\Microchip\TCPIP Stack\Objects - TCPIP Demo App-C32\TCP.o
 .debug_aranges
                0x00000280       0x20 ..\Microchip\TCPIP Stack\Objects - TCPIP Demo App-C32\Tick.o
 .debug_aranges
                0x000002a0       0x20 ..\Microchip\TCPIP Stack\Objects - TCPIP Demo App-C32\UDP.o
 .debug_aranges
                0x000002c0       0x20 Objects - TCPIP Demo App-C32\SMTPDemo.o
 .debug_aranges
                0x000002e0       0x28 C:/Program Files/Microchip/MPLAB C32/bin/../lib/gcc/pic32mx/3.4.4/../../../../pic32mx/lib/size\libc.a(strchr.o)
 .debug_aranges
                0x00000308       0x28 C:/Program Files/Microchip/MPLAB C32/bin/../lib/gcc/pic32mx/3.4.4/../../../../pic32mx/lib/size\libc.a(strstr.o)
 .debug_aranges
                0x00000330       0x28 C:/Program Files/Microchip/MPLAB C32/bin/../lib/gcc/pic32mx/3.4.4/../../../../pic32mx/lib/size\libc.a(exit.o)
 .debug_aranges
                0x00000358       0x38 C:/Program Files/Microchip/MPLAB C32/bin/../lib/gcc/pic32mx/3.4.4/../../../../pic32mx/lib/size\libc.a(rand.o)
 .debug_aranges
                0x00000390       0x28 C:/Program Files/Microchip/MPLAB C32/bin/../lib/gcc/pic32mx/3.4.4/../../../../pic32mx/lib/size\libc.a(atol.o)
 .debug_aranges
                0x000003b8       0x28 C:/Program Files/Microchip/MPLAB C32/bin/../lib/gcc/pic32mx/3.4.4/../../../../pic32mx/lib/size\libc.a(atoi.o)
 .debug_aranges
                0x000003e0       0x28 C:/Program Files/Microchip/MPLAB C32/bin/../lib/gcc/pic32mx/3.4.4/../../../../pic32mx/lib/size\libc.a(strtol.o)
 .debug_aranges
                0x00000408       0x48 C:/Program Files/Microchip/MPLAB C32/bin/../lib/gcc/pic32mx/3.4.4/../../../../pic32mx/lib/size\libc.a(_iobfuncs.o)
 .debug_aranges
                0x00000450       0xd0 C:/Program Files/Microchip/MPLAB C32/bin/../lib/gcc/pic32mx/3.4.4/../../../../pic32mx/lib/size\libc.a(stubs.o)
 .debug_aranges
                0x00000520       0x28 C:/Program Files/Microchip/MPLAB C32/bin/../lib/gcc/pic32mx/3.4.4/../../../../pic32mx/lib/size\libc.a(default-bootstrap-exception-handler.o)
 .debug_aranges
                0x00000548       0x28 C:/Program Files/Microchip/MPLAB C32/bin/../lib/gcc/pic32mx/3.4.4/../../../../pic32mx/lib/size\libc.a(default-on-reset.o)
 .debug_aranges
                0x00000570       0x28 C:/Program Files/Microchip/MPLAB C32/bin/../lib/gcc/pic32mx/3.4.4/../../../../pic32mx/lib/size\libc.a(default-on-bootstrap.o)
 .debug_aranges
                0x00000598       0x28 C:/Program Files/Microchip/MPLAB C32/bin/../lib/gcc/pic32mx/3.4.4/../../../../pic32mx/lib/size\libc.a(_mon_getc.o)
 .debug_aranges
                0x000005c0       0x28 C:/Program Files/Microchip/MPLAB C32/bin/../lib/gcc/pic32mx/3.4.4/../../../../pic32mx/lib/size\libc.a(_mon_write.o)
 .debug_aranges
                0x000005e8       0x28 C:/Program Files/Microchip/MPLAB C32/bin/../lib/gcc/pic32mx/3.4.4/../../../../pic32mx/lib/size\libc.a(_exit.o)
 .debug_aranges
                0x00000610       0x28 C:/Program Files/Microchip/MPLAB C32/bin/../lib/gcc/pic32mx/3.4.4/../../../../pic32mx/lib/size\libc.a(_mon_putc.o)
 .debug_aranges
                0x00000638       0x28 C:/Program Files/Microchip/MPLAB C32/bin/../lib/gcc/pic32mx/3.4.4/../../../../pic32mx/lib/size\libmchp_peripheral.a(int_disable_interrupts_lib.o)
 .debug_aranges
                0x00000660       0x28 C:/Program Files/Microchip/MPLAB C32/bin/../lib/gcc/pic32mx/3.4.4/../../../../pic32mx/lib/size\libmchp_peripheral.a(int_enable_mv_int_lib.o)
 .debug_aranges
                0x00000688       0x28 C:/Program Files/Microchip/MPLAB C32/bin/../lib/gcc/pic32mx/3.4.4/../../../../pic32mx/lib/size\libmchp_peripheral.a(int_restore_interrupts_lib.o)
 .debug_aranges
                0x000006b0       0x28 C:/Program Files/Microchip/MPLAB C32/bin/../lib/gcc/pic32mx/3.4.4/../../../../pic32mx/lib/size\libmchp_peripheral.a(soft_reset_lib.o)
 .debug_aranges
                0x000006d8       0x30 C:/Program Files/Microchip/MPLAB C32/bin/../lib/gcc/pic32mx/3.4.4/../../../../pic32mx/lib/size\libmchp_peripheral.a(pcache.o)
 .debug_aranges
                0x00000708       0x28 C:/Program Files/Microchip/MPLAB C32/bin/../lib/gcc/pic32mx/3.4.4/../../../../pic32mx/lib/size\libmchp_peripheral.a(int_enable_interrupts_lib.o)

.debug_pubnames
                0x00000000     0x141e
 *(.debug_pubnames)
 .debug_pubnames
                0x00000000       0x8c Objects - TCPIP Demo App-C32\MainDemo.o
 .debug_pubnames
                0x0000008c       0x9e Objects - TCPIP Demo App-C32\CustomHTTPApp.o
 .debug_pubnames
                0x0000012a       0x4e ..\Microchip\TCPIP Stack\Objects - TCPIP Demo App-C32\ARP.o
 .debug_pubnames
                0x00000178       0x2c ..\Microchip\TCPIP Stack\Objects - TCPIP Demo App-C32\Delay.o
 .debug_pubnames
                0x000001a4       0x7c ..\Microchip\TCPIP Stack\Objects - TCPIP Demo App-C32\DHCP.o
 .debug_pubnames
                0x00000220       0x3c ..\Microchip\TCPIP Stack\Objects - TCPIP Demo App-C32\DHCPs.o
 .debug_pubnames
                0x0000025c       0x55 ..\Microchip\TCPIP Stack\Objects - TCPIP Demo App-C32\DNS.o
 .debug_pubnames
                0x000002b1       0x9f ..\Microchip\TCPIP Stack\Objects - TCPIP Demo App-C32\DynDNS.o
 .debug_pubnames
                0x00000350      0x1b8 ..\Microchip\TCPIP Stack\Objects - TCPIP Demo App-C32\ENC28J60.o
 .debug_pubnames
                0x00000508       0x62 ..\Microchip\TCPIP Stack\Objects - TCPIP Demo App-C32\Hashes.o
 .debug_pubnames
                0x0000056a       0xfe ..\Microchip\TCPIP Stack\Objects - TCPIP Demo App-C32\Helpers.o
 .debug_pubnames
                0x00000668       0xcf ..\Microchip\TCPIP Stack\Objects - TCPIP Demo App-C32\HTTP2.o
 .debug_pubnames
                0x00000737       0x22 ..\Microchip\TCPIP Stack\Objects - TCPIP Demo App-C32\ICMP.o
 .debug_pubnames
                0x00000759       0x44 ..\Microchip\TCPIP Stack\Objects - TCPIP Demo App-C32\IP.o
 .debug_pubnames
                0x0000079d       0x45 ..\Microchip\TCPIP Stack\Objects - TCPIP Demo App-C32\LCDBlocking.o
 .debug_pubnames
                0x000007e2      0x140 ..\Microchip\TCPIP Stack\Objects - TCPIP Demo App-C32\MPFS2.o
 .debug_pubnames
                0x00000922       0x1f ..\Microchip\TCPIP Stack\Objects - TCPIP Demo App-C32\NBNS.o
 .debug_pubnames
                0x00000941       0xd2 ..\Microchip\TCPIP Stack\Objects - TCPIP Demo App-C32\SMTP.o
 .debug_pubnames
                0x00000a13       0x53 ..\Microchip\TCPIP Stack\Objects - TCPIP Demo App-C32\StackTsk.o
 .debug_pubnames
                0x00000a66      0x190 ..\Microchip\TCPIP Stack\Objects - TCPIP Demo App-C32\TCP.o
 .debug_pubnames
                0x00000bf6       0x7e ..\Microchip\TCPIP Stack\Objects - TCPIP Demo App-C32\Tick.o
 .debug_pubnames
                0x00000c74      0x143 ..\Microchip\TCPIP Stack\Objects - TCPIP Demo App-C32\UDP.o
 .debug_pubnames
                0x00000db7       0x1f Objects - TCPIP Demo App-C32\SMTPDemo.o
 .debug_pubnames
                0x00000dd6       0x21 Objects - TCPIP Demo App-C32\MPFSImg2-C32.o
 .debug_pubnames
                0x00000df7       0x1d C:/Program Files/Microchip/MPLAB C32/bin/../lib/gcc/pic32mx/3.4.4/../../../../pic32mx/lib/size\libc.a(strchr.o)
 .debug_pubnames
                0x00000e14       0x1d C:/Program Files/Microchip/MPLAB C32/bin/../lib/gcc/pic32mx/3.4.4/../../../../pic32mx/lib/size\libc.a(strstr.o)
 .debug_pubnames
                0x00000e31       0x1b C:/Program Files/Microchip/MPLAB C32/bin/../lib/gcc/pic32mx/3.4.4/../../../../pic32mx/lib/size\libc.a(exit.o)
 .debug_pubnames
                0x00000e4c       0x30 C:/Program Files/Microchip/MPLAB C32/bin/../lib/gcc/pic32mx/3.4.4/../../../../pic32mx/lib/size\libc.a(rand.o)
 .debug_pubnames
                0x00000e7c       0x1b C:/Program Files/Microchip/MPLAB C32/bin/../lib/gcc/pic32mx/3.4.4/../../../../pic32mx/lib/size\libc.a(atol.o)
 .debug_pubnames
                0x00000e97       0x1b C:/Program Files/Microchip/MPLAB C32/bin/../lib/gcc/pic32mx/3.4.4/../../../../pic32mx/lib/size\libc.a(atoi.o)
 .debug_pubnames
                0x00000eb2       0x1d C:/Program Files/Microchip/MPLAB C32/bin/../lib/gcc/pic32mx/3.4.4/../../../../pic32mx/lib/size\libc.a(strtol.o)
 .debug_pubnames
                0x00000ecf       0x70 C:/Program Files/Microchip/MPLAB C32/bin/../lib/gcc/pic32mx/3.4.4/../../../../pic32mx/lib/size\libc.a(_iobfuncs.o)
 .debug_pubnames
                0x00000f3f      0x2da C:/Program Files/Microchip/MPLAB C32/bin/../lib/gcc/pic32mx/3.4.4/../../../../pic32mx/lib/size\libc.a(stubs.o)
 .debug_pubnames
                0x00001219       0x33 C:/Program Files/Microchip/MPLAB C32/bin/../lib/gcc/pic32mx/3.4.4/../../../../pic32mx/lib/size\libc.a(default-bootstrap-exception-handler.o)
 .debug_pubnames
                0x0000124c       0x20 C:/Program Files/Microchip/MPLAB C32/bin/../lib/gcc/pic32mx/3.4.4/../../../../pic32mx/lib/size\libc.a(default-on-reset.o)
 .debug_pubnames
                0x0000126c       0x24 C:/Program Files/Microchip/MPLAB C32/bin/../lib/gcc/pic32mx/3.4.4/../../../../pic32mx/lib/size\libc.a(default-on-bootstrap.o)
 .debug_pubnames
                0x00001290       0x20 C:/Program Files/Microchip/MPLAB C32/bin/../lib/gcc/pic32mx/3.4.4/../../../../pic32mx/lib/size\libc.a(_mon_getc.o)
 .debug_pubnames
                0x000012b0       0x21 C:/Program Files/Microchip/MPLAB C32/bin/../lib/gcc/pic32mx/3.4.4/../../../../pic32mx/lib/size\libc.a(_mon_write.o)
 .debug_pubnames
                0x000012d1       0x1c C:/Program Files/Microchip/MPLAB C32/bin/../lib/gcc/pic32mx/3.4.4/../../../../pic32mx/lib/size\libc.a(_exit.o)
 .debug_pubnames
                0x000012ed       0x20 C:/Program Files/Microchip/MPLAB C32/bin/../lib/gcc/pic32mx/3.4.4/../../../../pic32mx/lib/size\libc.a(_mon_putc.o)
 .debug_pubnames
                0x0000130d       0x2b C:/Program Files/Microchip/MPLAB C32/bin/../lib/gcc/pic32mx/3.4.4/../../../../pic32mx/lib/size\libmchp_peripheral.a(int_disable_interrupts_lib.o)
 .debug_pubnames
                0x00001338       0x36 C:/Program Files/Microchip/MPLAB C32/bin/../lib/gcc/pic32mx/3.4.4/../../../../pic32mx/lib/size\libmchp_peripheral.a(int_enable_mv_int_lib.o)
 .debug_pubnames
                0x0000136e       0x2b C:/Program Files/Microchip/MPLAB C32/bin/../lib/gcc/pic32mx/3.4.4/../../../../pic32mx/lib/size\libmchp_peripheral.a(int_restore_interrupts_lib.o)
 .debug_pubnames
                0x00001399       0x20 C:/Program Files/Microchip/MPLAB C32/bin/../lib/gcc/pic32mx/3.4.4/../../../../pic32mx/lib/size\libmchp_peripheral.a(soft_reset_lib.o)
 .debug_pubnames
                0x000013b9       0x3b C:/Program Files/Microchip/MPLAB C32/bin/../lib/gcc/pic32mx/3.4.4/../../../../pic32mx/lib/size\libmchp_peripheral.a(pcache.o)
 .debug_pubnames
                0x000013f4       0x2a C:/Program Files/Microchip/MPLAB C32/bin/../lib/gcc/pic32mx/3.4.4/../../../../pic32mx/lib/size\libmchp_peripheral.a(int_enable_interrupts_lib.o)

.debug_info     0x00000000    0x1dc42
 *(.debug_info .gnu.linkonce.wi.*)
 .debug_info    0x00000000     0x12bc Objects - TCPIP Demo App-C32\MainDemo.o
 .debug_info    0x000012bc      0x87d Objects - TCPIP Demo App-C32\CustomHTTPApp.o
 .debug_info    0x00001b39      0x397 ..\Microchip\TCPIP Stack\Objects - TCPIP Demo App-C32\UDPPerformanceTest.o
 .debug_info    0x00001ed0      0x38d ..\Microchip\TCPIP Stack\Objects - TCPIP Demo App-C32\Announce.o
 .debug_info    0x0000225d      0xd09 ..\Microchip\TCPIP Stack\Objects - TCPIP Demo App-C32\ARP.o
 .debug_info    0x00002f66      0x41d ..\Microchip\TCPIP Stack\Objects - TCPIP Demo App-C32\Delay.o
 .debug_info    0x00003383     0x109d ..\Microchip\TCPIP Stack\Objects - TCPIP Demo App-C32\DHCP.o
 .debug_info    0x00004420      0xe55 ..\Microchip\TCPIP Stack\Objects - TCPIP Demo App-C32\DHCPs.o
 .debug_info    0x00005275      0xfc9 ..\Microchip\TCPIP Stack\Objects - TCPIP Demo App-C32\DNS.o
 .debug_info    0x0000623e     0x1114 ..\Microchip\TCPIP Stack\Objects - TCPIP Demo App-C32\DynDNS.o
 .debug_info    0x00007352     0x29cb ..\Microchip\TCPIP Stack\Objects - TCPIP Demo App-C32\ENC28J60.o
 .debug_info    0x00009d1d      0x388 ..\Microchip\TCPIP Stack\Objects - TCPIP Demo App-C32\FTP.o
 .debug_info    0x0000a0a5      0x76b ..\Microchip\TCPIP Stack\Objects - TCPIP Demo App-C32\Hashes.o
 .debug_info    0x0000a810      0xfe4 ..\Microchip\TCPIP Stack\Objects - TCPIP Demo App-C32\Helpers.o
 .debug_info    0x0000b7f4     0x10e4 ..\Microchip\TCPIP Stack\Objects - TCPIP Demo App-C32\HTTP2.o
 .debug_info    0x0000c8d8      0x389 ..\Microchip\TCPIP Stack\Objects - TCPIP Demo App-C32\HTTP.o
 .debug_info    0x0000cc61      0x957 ..\Microchip\TCPIP Stack\Objects - TCPIP Demo App-C32\ICMP.o
 .debug_info    0x0000d5b8      0xd37 ..\Microchip\TCPIP Stack\Objects - TCPIP Demo App-C32\IP.o
 .debug_info    0x0000e2ef      0x579 ..\Microchip\TCPIP Stack\Objects - TCPIP Demo App-C32\LCDBlocking.o
 .debug_info    0x0000e868      0xb39 ..\Microchip\TCPIP Stack\Objects - TCPIP Demo App-C32\MPFS2.o
 .debug_info    0x0000f3a1      0x389 ..\Microchip\TCPIP Stack\Objects - TCPIP Demo App-C32\MPFS.o
 .debug_info    0x0000f72a      0xd48 ..\Microchip\TCPIP Stack\Objects - TCPIP Demo App-C32\NBNS.o
 .debug_info    0x00010472      0x38b ..\Microchip\TCPIP Stack\Objects - TCPIP Demo App-C32\Reboot.o
 .debug_info    0x000107fd     0x163a ..\Microchip\TCPIP Stack\Objects - TCPIP Demo App-C32\SMTP.o
 .debug_info    0x00011e37      0x389 ..\Microchip\TCPIP Stack\Objects - TCPIP Demo App-C32\SNMP.o
 .debug_info    0x000121c0      0x389 ..\Microchip\TCPIP Stack\Objects - TCPIP Demo App-C32\SNTP.o
 .debug_info    0x00012549      0x38e ..\Microchip\TCPIP Stack\Objects - TCPIP Demo App-C32\SPIEEPROM.o
 .debug_info    0x000128d7      0x38d ..\Microchip\TCPIP Stack\Objects - TCPIP Demo App-C32\SPIFlash.o
 .debug_info    0x00012c64      0x38b ..\Microchip\TCPIP Stack\Objects - TCPIP Demo App-C32\SPIRAM.o
 .debug_info    0x00012fef      0xc7d ..\Microchip\TCPIP Stack\Objects - TCPIP Demo App-C32\StackTsk.o
 .debug_info    0x00013c6c     0x2284 ..\Microchip\TCPIP Stack\Objects - TCPIP Demo App-C32\TCP.o
 .debug_info    0x00015ef0      0x397 ..\Microchip\TCPIP Stack\Objects - TCPIP Demo App-C32\TCPPerformanceTest.o
 .debug_info    0x00016287      0x38b ..\Microchip\TCPIP Stack\Objects - TCPIP Demo App-C32\Telnet.o
 .debug_info    0x00016612      0x38a ..\Microchip\TCPIP Stack\Objects - TCPIP Demo App-C32\TFTPc.o
 .debug_info    0x0001699c      0xb17 ..\Microchip\TCPIP Stack\Objects - TCPIP Demo App-C32\Tick.o
 .debug_info    0x000174b3      0x393 ..\Microchip\TCPIP Stack\Objects - TCPIP Demo App-C32\UART2TCPBridge.o
 .debug_info    0x00017846      0x389 ..\Microchip\TCPIP Stack\Objects - TCPIP Demo App-C32\UART.o
 .debug_info    0x00017bcf     0x1236 ..\Microchip\TCPIP Stack\Objects - TCPIP Demo App-C32\UDP.o
 .debug_info    0x00018e05      0x386 Objects - TCPIP Demo App-C32\CustomSNMPApp.o
 .debug_info    0x0001918b      0x383 Objects - TCPIP Demo App-C32\UARTConfig.o
 .debug_info    0x0001950e      0x389 Objects - TCPIP Demo App-C32\GenericTCPClient.o
 .debug_info    0x00019897      0x389 Objects - TCPIP Demo App-C32\GenericTCPServer.o
 .debug_info    0x00019c20      0x386 Objects - TCPIP Demo App-C32\LegacyHTTPApp.o
 .debug_info    0x00019fa6      0x381 Objects - TCPIP Demo App-C32\PingDemo.o
 .debug_info    0x0001a327      0x83d Objects - TCPIP Demo App-C32\SMTPDemo.o
 .debug_info    0x0001ab64      0x390 ..\Microchip\TCPIP Stack\Objects - TCPIP Demo App-C32\BerkeleyAPI.o
 .debug_info    0x0001aef4      0x38e Objects - TCPIP Demo App-C32\BerkeleyUDPClientDemo.o
 .debug_info    0x0001b282      0x38e Objects - TCPIP Demo App-C32\BerkeleyTCPClientDemo.o
 .debug_info    0x0001b610      0x38e Objects - TCPIP Demo App-C32\BerkeleyTCPServerDemo.o
 .debug_info    0x0001b99e      0x38f ..\Microchip\TCPIP Stack\Objects - TCPIP Demo App-C32\ENCX24J600.o
 .debug_info    0x0001bd2d      0x38b ..\Microchip\TCPIP Stack\Objects - TCPIP Demo App-C32\Random.o
 .debug_info    0x0001c0b8      0x388 ..\Microchip\TCPIP Stack\Objects - TCPIP Demo App-C32\RSA.o
 .debug_info    0x0001c440      0x388 ..\Microchip\TCPIP Stack\Objects - TCPIP Demo App-C32\SSL.o
 .debug_info    0x0001c7c8      0x38c ..\Microchip\TCPIP Stack\Objects - TCPIP Demo App-C32\ARCFOUR.o
 .debug_info    0x0001cb54      0x38b ..\Microchip\TCPIP Stack\Objects - TCPIP Demo App-C32\BigInt.o
 .debug_info    0x0001cedf      0x386 Objects - TCPIP Demo App-C32\CustomSSLCert.o
 .debug_info    0x0001d265      0x3c5 Objects - TCPIP Demo App-C32\MPFSImg2-C32.o
 .debug_info    0x0001d62a       0x30 C:/Program Files/Microchip/MPLAB C32/bin/../lib/gcc/pic32mx/3.4.4/../../../../pic32mx/lib/size\libc.a(strchr.o)
 .debug_info    0x0001d65a       0x30 C:/Program Files/Microchip/MPLAB C32/bin/../lib/gcc/pic32mx/3.4.4/../../../../pic32mx/lib/size\libc.a(strstr.o)
 .debug_info    0x0001d68a       0x30 C:/Program Files/Microchip/MPLAB C32/bin/../lib/gcc/pic32mx/3.4.4/../../../../pic32mx/lib/size\libc.a(exit.o)
 .debug_info    0x0001d6ba       0x54 C:/Program Files/Microchip/MPLAB C32/bin/../lib/gcc/pic32mx/3.4.4/../../../../pic32mx/lib/size\libc.a(rand.o)
 .debug_info    0x0001d70e       0x30 C:/Program Files/Microchip/MPLAB C32/bin/../lib/gcc/pic32mx/3.4.4/../../../../pic32mx/lib/size\libc.a(atol.o)
 .debug_info    0x0001d73e       0x30 C:/Program Files/Microchip/MPLAB C32/bin/../lib/gcc/pic32mx/3.4.4/../../../../pic32mx/lib/size\libc.a(atoi.o)
 .debug_info    0x0001d76e       0x30 C:/Program Files/Microchip/MPLAB C32/bin/../lib/gcc/pic32mx/3.4.4/../../../../pic32mx/lib/size\libc.a(strtol.o)
 .debug_info    0x0001d79e       0x78 C:/Program Files/Microchip/MPLAB C32/bin/../lib/gcc/pic32mx/3.4.4/../../../../pic32mx/lib/size\libc.a(_iobfuncs.o)
 .debug_info    0x0001d816      0x1aa C:/Program Files/Microchip/MPLAB C32/bin/../lib/gcc/pic32mx/3.4.4/../../../../pic32mx/lib/size\libc.a(stubs.o)
 .debug_info    0x0001d9c0       0x30 C:/Program Files/Microchip/MPLAB C32/bin/../lib/gcc/pic32mx/3.4.4/../../../../pic32mx/lib/size\libc.a(default-bootstrap-exception-handler.o)
 .debug_info    0x0001d9f0       0x30 C:/Program Files/Microchip/MPLAB C32/bin/../lib/gcc/pic32mx/3.4.4/../../../../pic32mx/lib/size\libc.a(default-on-reset.o)
 .debug_info    0x0001da20       0x30 C:/Program Files/Microchip/MPLAB C32/bin/../lib/gcc/pic32mx/3.4.4/../../../../pic32mx/lib/size\libc.a(default-on-bootstrap.o)
 .debug_info    0x0001da50       0x30 C:/Program Files/Microchip/MPLAB C32/bin/../lib/gcc/pic32mx/3.4.4/../../../../pic32mx/lib/size\libc.a(_mon_getc.o)
 .debug_info    0x0001da80       0x30 C:/Program Files/Microchip/MPLAB C32/bin/../lib/gcc/pic32mx/3.4.4/../../../../pic32mx/lib/size\libc.a(_mon_write.o)
 .debug_info    0x0001dab0       0x30 C:/Program Files/Microchip/MPLAB C32/bin/../lib/gcc/pic32mx/3.4.4/../../../../pic32mx/lib/size\libc.a(_exit.o)
 .debug_info    0x0001dae0       0x30 C:/Program Files/Microchip/MPLAB C32/bin/../lib/gcc/pic32mx/3.4.4/../../../../pic32mx/lib/size\libc.a(_mon_putc.o)
 .debug_info    0x0001db10       0x30 C:/Program Files/Microchip/MPLAB C32/bin/../lib/gcc/pic32mx/3.4.4/../../../../pic32mx/lib/size\libmchp_peripheral.a(int_disable_interrupts_lib.o)
 .debug_info    0x0001db40       0x30 C:/Program Files/Microchip/MPLAB C32/bin/../lib/gcc/pic32mx/3.4.4/../../../../pic32mx/lib/size\libmchp_peripheral.a(int_enable_mv_int_lib.o)
 .debug_info    0x0001db70       0x30 C:/Program Files/Microchip/MPLAB C32/bin/../lib/gcc/pic32mx/3.4.4/../../../../pic32mx/lib/size\libmchp_peripheral.a(int_restore_interrupts_lib.o)
 .debug_info    0x0001dba0       0x30 C:/Program Files/Microchip/MPLAB C32/bin/../lib/gcc/pic32mx/3.4.4/../../../../pic32mx/lib/size\libmchp_peripheral.a(soft_reset_lib.o)
 .debug_info    0x0001dbd0       0x42 C:/Program Files/Microchip/MPLAB C32/bin/../lib/gcc/pic32mx/3.4.4/../../../../pic32mx/lib/size\libmchp_peripheral.a(pcache.o)
 .debug_info    0x0001dc12       0x30 C:/Program Files/Microchip/MPLAB C32/bin/../lib/gcc/pic32mx/3.4.4/../../../../pic32mx/lib/size\libmchp_peripheral.a(int_enable_interrupts_lib.o)

.debug_abbrev   0x00000000     0x45b0
 *(.debug_abbrev)
 .debug_abbrev  0x00000000      0x2d5 Objects - TCPIP Demo App-C32\MainDemo.o
 .debug_abbrev  0x000002d5      0x14f Objects - TCPIP Demo App-C32\CustomHTTPApp.o
 .debug_abbrev  0x00000424       0xab ..\Microchip\TCPIP Stack\Objects - TCPIP Demo App-C32\UDPPerformanceTest.o
 .debug_abbrev  0x000004cf       0xab ..\Microchip\TCPIP Stack\Objects - TCPIP Demo App-C32\Announce.o
 .debug_abbrev  0x0000057a      0x23a ..\Microchip\TCPIP Stack\Objects - TCPIP Demo App-C32\ARP.o
 .debug_abbrev  0x000007b4       0xe0 ..\Microchip\TCPIP Stack\Objects - TCPIP Demo App-C32\Delay.o
 .debug_abbrev  0x00000894      0x1e1 ..\Microchip\TCPIP Stack\Objects - TCPIP Demo App-C32\DHCP.o
 .debug_abbrev  0x00000a75      0x1ba ..\Microchip\TCPIP Stack\Objects - TCPIP Demo App-C32\DHCPs.o
 .debug_abbrev  0x00000c2f      0x200 ..\Microchip\TCPIP Stack\Objects - TCPIP Demo App-C32\DNS.o
 .debug_abbrev  0x00000e2f      0x21b ..\Microchip\TCPIP Stack\Objects - TCPIP Demo App-C32\DynDNS.o
 .debug_abbrev  0x0000104a      0x2ce ..\Microchip\TCPIP Stack\Objects - TCPIP Demo App-C32\ENC28J60.o
 .debug_abbrev  0x00001318       0xab ..\Microchip\TCPIP Stack\Objects - TCPIP Demo App-C32\FTP.o
 .debug_abbrev  0x000013c3      0x1ad ..\Microchip\TCPIP Stack\Objects - TCPIP Demo App-C32\Hashes.o
 .debug_abbrev  0x00001570      0x1c0 ..\Microchip\TCPIP Stack\Objects - TCPIP Demo App-C32\Helpers.o
 .debug_abbrev  0x00001730      0x241 ..\Microchip\TCPIP Stack\Objects - TCPIP Demo App-C32\HTTP2.o
 .debug_abbrev  0x00001971       0xab ..\Microchip\TCPIP Stack\Objects - TCPIP Demo App-C32\HTTP.o
 .debug_abbrev  0x00001a1c      0x157 ..\Microchip\TCPIP Stack\Objects - TCPIP Demo App-C32\ICMP.o
 .debug_abbrev  0x00001b73      0x1bb ..\Microchip\TCPIP Stack\Objects - TCPIP Demo App-C32\IP.o
 .debug_abbrev  0x00001d2e      0x153 ..\Microchip\TCPIP Stack\Objects - TCPIP Demo App-C32\LCDBlocking.o
 .debug_abbrev  0x00001e81      0x20d ..\Microchip\TCPIP Stack\Objects - TCPIP Demo App-C32\MPFS2.o
 .debug_abbrev  0x0000208e       0xab ..\Microchip\TCPIP Stack\Objects - TCPIP Demo App-C32\MPFS.o
 .debug_abbrev  0x00002139      0x1a2 ..\Microchip\TCPIP Stack\Objects - TCPIP Demo App-C32\NBNS.o
 .debug_abbrev  0x000022db       0xab ..\Microchip\TCPIP Stack\Objects - TCPIP Demo App-C32\Reboot.o
 .debug_abbrev  0x00002386      0x2a5 ..\Microchip\TCPIP Stack\Objects - TCPIP Demo App-C32\SMTP.o
 .debug_abbrev  0x0000262b       0xab ..\Microchip\TCPIP Stack\Objects - TCPIP Demo App-C32\SNMP.o
 .debug_abbrev  0x000026d6       0xab ..\Microchip\TCPIP Stack\Objects - TCPIP Demo App-C32\SNTP.o
 .debug_abbrev  0x00002781       0xab ..\Microchip\TCPIP Stack\Objects - TCPIP Demo App-C32\SPIEEPROM.o
 .debug_abbrev  0x0000282c       0xab ..\Microchip\TCPIP Stack\Objects - TCPIP Demo App-C32\SPIFlash.o
 .debug_abbrev  0x000028d7       0xab ..\Microchip\TCPIP Stack\Objects - TCPIP Demo App-C32\SPIRAM.o
 .debug_abbrev  0x00002982      0x192 ..\Microchip\TCPIP Stack\Objects - TCPIP Demo App-C32\StackTsk.o
 .debug_abbrev  0x00002b14      0x269 ..\Microchip\TCPIP Stack\Objects - TCPIP Demo App-C32\TCP.o
 .debug_abbrev  0x00002d7d       0xab ..\Microchip\TCPIP Stack\Objects - TCPIP Demo App-C32\TCPPerformanceTest.o
 .debug_abbrev  0x00002e28       0xab ..\Microchip\TCPIP Stack\Objects - TCPIP Demo App-C32\Telnet.o
 .debug_abbrev  0x00002ed3       0xab ..\Microchip\TCPIP Stack\Objects - TCPIP Demo App-C32\TFTPc.o
 .debug_abbrev  0x00002f7e      0x1c8 ..\Microchip\TCPIP Stack\Objects - TCPIP Demo App-C32\Tick.o
 .debug_abbrev  0x00003146       0xab ..\Microchip\TCPIP Stack\Objects - TCPIP Demo App-C32\UART2TCPBridge.o
 .debug_abbrev  0x000031f1       0xab ..\Microchip\TCPIP Stack\Objects - TCPIP Demo App-C32\UART.o
 .debug_abbrev  0x0000329c      0x25e ..\Microchip\TCPIP Stack\Objects - TCPIP Demo App-C32\UDP.o
 .debug_abbrev  0x000034fa       0xab Objects - TCPIP Demo App-C32\CustomSNMPApp.o
 .debug_abbrev  0x000035a5       0xab Objects - TCPIP Demo App-C32\UARTConfig.o
 .debug_abbrev  0x00003650       0xab Objects - TCPIP Demo App-C32\GenericTCPClient.o
 .debug_abbrev  0x000036fb       0xab Objects - TCPIP Demo App-C32\GenericTCPServer.o
 .debug_abbrev  0x000037a6       0xab Objects - TCPIP Demo App-C32\LegacyHTTPApp.o
 .debug_abbrev  0x00003851       0xab Objects - TCPIP Demo App-C32\PingDemo.o
 .debug_abbrev  0x000038fc      0x181 Objects - TCPIP Demo App-C32\SMTPDemo.o
 .debug_abbrev  0x00003a7d       0xab ..\Microchip\TCPIP Stack\Objects - TCPIP Demo App-C32\BerkeleyAPI.o
 .debug_abbrev  0x00003b28       0xab Objects - TCPIP Demo App-C32\BerkeleyUDPClientDemo.o
 .debug_abbrev  0x00003bd3       0xab Objects - TCPIP Demo App-C32\BerkeleyTCPClientDemo.o
 .debug_abbrev  0x00003c7e       0xab Objects - TCPIP Demo App-C32\BerkeleyTCPServerDemo.o
 .debug_abbrev  0x00003d29       0xab ..\Microchip\TCPIP Stack\Objects - TCPIP Demo App-C32\ENCX24J600.o
 .debug_abbrev  0x00003dd4       0xab ..\Microchip\TCPIP Stack\Objects - TCPIP Demo App-C32\Random.o
 .debug_abbrev  0x00003e7f       0xab ..\Microchip\TCPIP Stack\Objects - TCPIP Demo App-C32\RSA.o
 .debug_abbrev  0x00003f2a       0xab ..\Microchip\TCPIP Stack\Objects - TCPIP Demo App-C32\SSL.o
 .debug_abbrev  0x00003fd5       0xab ..\Microchip\TCPIP Stack\Objects - TCPIP Demo App-C32\ARCFOUR.o
 .debug_abbrev  0x00004080       0xab ..\Microchip\TCPIP Stack\Objects - TCPIP Demo App-C32\BigInt.o
 .debug_abbrev  0x0000412b       0xab Objects - TCPIP Demo App-C32\CustomSSLCert.o
 .debug_abbrev  0x000041d6       0xd5 Objects - TCPIP Demo App-C32\MPFSImg2-C32.o
 .debug_abbrev  0x000042ab       0x23 C:/Program Files/Microchip/MPLAB C32/bin/../lib/gcc/pic32mx/3.4.4/../../../../pic32mx/lib/size\libc.a(strchr.o)
 .debug_abbrev  0x000042ce       0x23 C:/Program Files/Microchip/MPLAB C32/bin/../lib/gcc/pic32mx/3.4.4/../../../../pic32mx/lib/size\libc.a(strstr.o)
 .debug_abbrev  0x000042f1       0x23 C:/Program Files/Microchip/MPLAB C32/bin/../lib/gcc/pic32mx/3.4.4/../../../../pic32mx/lib/size\libc.a(exit.o)
 .debug_abbrev  0x00004314       0x23 C:/Program Files/Microchip/MPLAB C32/bin/../lib/gcc/pic32mx/3.4.4/../../../../pic32mx/lib/size\libc.a(rand.o)
 .debug_abbrev  0x00004337       0x23 C:/Program Files/Microchip/MPLAB C32/bin/../lib/gcc/pic32mx/3.4.4/../../../../pic32mx/lib/size\libc.a(atol.o)
 .debug_abbrev  0x0000435a       0x23 C:/Program Files/Microchip/MPLAB C32/bin/../lib/gcc/pic32mx/3.4.4/../../../../pic32mx/lib/size\libc.a(atoi.o)
 .debug_abbrev  0x0000437d       0x23 C:/Program Files/Microchip/MPLAB C32/bin/../lib/gcc/pic32mx/3.4.4/../../../../pic32mx/lib/size\libc.a(strtol.o)
 .debug_abbrev  0x000043a0        0x1 C:/Program Files/Microchip/MPLAB C32/bin/../lib/gcc/pic32mx/3.4.4/../../../../pic32mx/lib/size\libc.a(_iobdata.o)
 .debug_abbrev  0x000043a1       0x23 C:/Program Files/Microchip/MPLAB C32/bin/../lib/gcc/pic32mx/3.4.4/../../../../pic32mx/lib/size\libc.a(_iobfuncs.o)
 .debug_abbrev  0x000043c4       0x23 C:/Program Files/Microchip/MPLAB C32/bin/../lib/gcc/pic32mx/3.4.4/../../../../pic32mx/lib/size\libc.a(stubs.o)
 .debug_abbrev  0x000043e7       0x23 C:/Program Files/Microchip/MPLAB C32/bin/../lib/gcc/pic32mx/3.4.4/../../../../pic32mx/lib/size\libc.a(default-bootstrap-exception-handler.o)
 .debug_abbrev  0x0000440a       0x23 C:/Program Files/Microchip/MPLAB C32/bin/../lib/gcc/pic32mx/3.4.4/../../../../pic32mx/lib/size\libc.a(default-on-reset.o)
 .debug_abbrev  0x0000442d       0x23 C:/Program Files/Microchip/MPLAB C32/bin/../lib/gcc/pic32mx/3.4.4/../../../../pic32mx/lib/size\libc.a(default-on-bootstrap.o)
 .debug_abbrev  0x00004450       0x23 C:/Program Files/Microchip/MPLAB C32/bin/../lib/gcc/pic32mx/3.4.4/../../../../pic32mx/lib/size\libc.a(_mon_getc.o)
 .debug_abbrev  0x00004473       0x23 C:/Program Files/Microchip/MPLAB C32/bin/../lib/gcc/pic32mx/3.4.4/../../../../pic32mx/lib/size\libc.a(_mon_write.o)
 .debug_abbrev  0x00004496       0x23 C:/Program Files/Microchip/MPLAB C32/bin/../lib/gcc/pic32mx/3.4.4/../../../../pic32mx/lib/size\libc.a(_exit.o)
 .debug_abbrev  0x000044b9        0x1 C:/Program Files/Microchip/MPLAB C32/bin/../lib/gcc/pic32mx/3.4.4/../../../../pic32mx/lib/size\libc.a(ctype.o)
 .debug_abbrev  0x000044ba        0x1 C:/Program Files/Microchip/MPLAB C32/bin/../lib/gcc/pic32mx/3.4.4/../../../../pic32mx/lib/size\libc.a(errno.o)
 .debug_abbrev  0x000044bb       0x23 C:/Program Files/Microchip/MPLAB C32/bin/../lib/gcc/pic32mx/3.4.4/../../../../pic32mx/lib/size\libc.a(_mon_putc.o)
 .debug_abbrev  0x000044de       0x23 C:/Program Files/Microchip/MPLAB C32/bin/../lib/gcc/pic32mx/3.4.4/../../../../pic32mx/lib/size\libmchp_peripheral.a(int_disable_interrupts_lib.o)
 .debug_abbrev  0x00004501       0x23 C:/Program Files/Microchip/MPLAB C32/bin/../lib/gcc/pic32mx/3.4.4/../../../../pic32mx/lib/size\libmchp_peripheral.a(int_enable_mv_int_lib.o)
 .debug_abbrev  0x00004524       0x23 C:/Program Files/Microchip/MPLAB C32/bin/../lib/gcc/pic32mx/3.4.4/../../../../pic32mx/lib/size\libmchp_peripheral.a(int_restore_interrupts_lib.o)
 .debug_abbrev  0x00004547       0x23 C:/Program Files/Microchip/MPLAB C32/bin/../lib/gcc/pic32mx/3.4.4/../../../../pic32mx/lib/size\libmchp_peripheral.a(soft_reset_lib.o)
 .debug_abbrev  0x0000456a       0x23 C:/Program Files/Microchip/MPLAB C32/bin/../lib/gcc/pic32mx/3.4.4/../../../../pic32mx/lib/size\libmchp_peripheral.a(pcache.o)
 .debug_abbrev  0x0000458d       0x23 C:/Program Files/Microchip/MPLAB C32/bin/../lib/gcc/pic32mx/3.4.4/../../../../pic32mx/lib/size\libmchp_peripheral.a(int_enable_interrupts_lib.o)

.debug_line     0x00000000     0x59ab
 *(.debug_line)
 .debug_line    0x00000000      0x341 Objects - TCPIP Demo App-C32\MainDemo.o
 .debug_line    0x00000341      0x1ba Objects - TCPIP Demo App-C32\CustomHTTPApp.o
 .debug_line    0x000004fb       0x90 ..\Microchip\TCPIP Stack\Objects - TCPIP Demo App-C32\UDPPerformanceTest.o
 .debug_line    0x0000058b       0x90 ..\Microchip\TCPIP Stack\Objects - TCPIP Demo App-C32\Announce.o
 .debug_line    0x0000061b      0x162 ..\Microchip\TCPIP Stack\Objects - TCPIP Demo App-C32\ARP.o
 .debug_line    0x0000077d       0xdd ..\Microchip\TCPIP Stack\Objects - TCPIP Demo App-C32\Delay.o
 .debug_line    0x0000085a      0x292 ..\Microchip\TCPIP Stack\Objects - TCPIP Demo App-C32\DHCP.o
 .debug_line    0x00000aec      0x1f2 ..\Microchip\TCPIP Stack\Objects - TCPIP Demo App-C32\DHCPs.o
 .debug_line    0x00000cde      0x241 ..\Microchip\TCPIP Stack\Objects - TCPIP Demo App-C32\DNS.o
 .debug_line    0x00000f1f      0x2b0 ..\Microchip\TCPIP Stack\Objects - TCPIP Demo App-C32\DynDNS.o
 .debug_line    0x000011cf      0x4b9 ..\Microchip\TCPIP Stack\Objects - TCPIP Demo App-C32\ENC28J60.o
 .debug_line    0x00001688       0x90 ..\Microchip\TCPIP Stack\Objects - TCPIP Demo App-C32\FTP.o
 .debug_line    0x00001718      0x18b ..\Microchip\TCPIP Stack\Objects - TCPIP Demo App-C32\Hashes.o
 .debug_line    0x000018a3      0x299 ..\Microchip\TCPIP Stack\Objects - TCPIP Demo App-C32\Helpers.o
 .debug_line    0x00001b3c      0x4e0 ..\Microchip\TCPIP Stack\Objects - TCPIP Demo App-C32\HTTP2.o
 .debug_line    0x0000201c       0x90 ..\Microchip\TCPIP Stack\Objects - TCPIP Demo App-C32\HTTP.o
 .debug_line    0x000020ac      0x109 ..\Microchip\TCPIP Stack\Objects - TCPIP Demo App-C32\ICMP.o
 .debug_line    0x000021b5      0x13e ..\Microchip\TCPIP Stack\Objects - TCPIP Demo App-C32\IP.o
 .debug_line    0x000022f3      0x158 ..\Microchip\TCPIP Stack\Objects - TCPIP Demo App-C32\LCDBlocking.o
 .debug_line    0x0000244b      0x2ba ..\Microchip\TCPIP Stack\Objects - TCPIP Demo App-C32\MPFS2.o
 .debug_line    0x00002705       0x90 ..\Microchip\TCPIP Stack\Objects - TCPIP Demo App-C32\MPFS.o
 .debug_line    0x00002795      0x183 ..\Microchip\TCPIP Stack\Objects - TCPIP Demo App-C32\NBNS.o
 .debug_line    0x00002918       0x90 ..\Microchip\TCPIP Stack\Objects - TCPIP Demo App-C32\Reboot.o
 .debug_line    0x000029a8      0x428 ..\Microchip\TCPIP Stack\Objects - TCPIP Demo App-C32\SMTP.o
 .debug_line    0x00002dd0       0x90 ..\Microchip\TCPIP Stack\Objects - TCPIP Demo App-C32\SNMP.o
 .debug_line    0x00002e60       0x90 ..\Microchip\TCPIP Stack\Objects - TCPIP Demo App-C32\SNTP.o
 .debug_line    0x00002ef0       0x90 ..\Microchip\TCPIP Stack\Objects - TCPIP Demo App-C32\SPIEEPROM.o
 .debug_line    0x00002f80       0x90 ..\Microchip\TCPIP Stack\Objects - TCPIP Demo App-C32\SPIFlash.o
 .debug_line    0x00003010       0x90 ..\Microchip\TCPIP Stack\Objects - TCPIP Demo App-C32\SPIRAM.o
 .debug_line    0x000030a0      0x158 ..\Microchip\TCPIP Stack\Objects - TCPIP Demo App-C32\StackTsk.o
 .debug_line    0x000031f8      0x97c ..\Microchip\TCPIP Stack\Objects - TCPIP Demo App-C32\TCP.o
 .debug_line    0x00003b74       0x90 ..\Microchip\TCPIP Stack\Objects - TCPIP Demo App-C32\TCPPerformanceTest.o
 .debug_line    0x00003c04       0x90 ..\Microchip\TCPIP Stack\Objects - TCPIP Demo App-C32\Telnet.o
 .debug_line    0x00003c94       0x90 ..\Microchip\TCPIP Stack\Objects - TCPIP Demo App-C32\TFTPc.o
 .debug_line    0x00003d24      0x11b ..\Microchip\TCPIP Stack\Objects - TCPIP Demo App-C32\Tick.o
 .debug_line    0x00003e3f       0x90 ..\Microchip\TCPIP Stack\Objects - TCPIP Demo App-C32\UART2TCPBridge.o
 .debug_line    0x00003ecf       0x90 ..\Microchip\TCPIP Stack\Objects - TCPIP Demo App-C32\UART.o
 .debug_line    0x00003f5f      0x237 ..\Microchip\TCPIP Stack\Objects - TCPIP Demo App-C32\UDP.o
 .debug_line    0x00004196       0x90 Objects - TCPIP Demo App-C32\CustomSNMPApp.o
 .debug_line    0x00004226       0x90 Objects - TCPIP Demo App-C32\UARTConfig.o
 .debug_line    0x000042b6       0x90 Objects - TCPIP Demo App-C32\GenericTCPClient.o
 .debug_line    0x00004346       0x90 Objects - TCPIP Demo App-C32\GenericTCPServer.o
 .debug_line    0x000043d6       0x90 Objects - TCPIP Demo App-C32\LegacyHTTPApp.o
 .debug_line    0x00004466       0x90 Objects - TCPIP Demo App-C32\PingDemo.o
 .debug_line    0x000044f6      0x14a Objects - TCPIP Demo App-C32\SMTPDemo.o
 .debug_line    0x00004640       0x90 ..\Microchip\TCPIP Stack\Objects - TCPIP Demo App-C32\BerkeleyAPI.o
 .debug_line    0x000046d0       0x90 Objects - TCPIP Demo App-C32\BerkeleyUDPClientDemo.o
 .debug_line    0x00004760       0x90 Objects - TCPIP Demo App-C32\BerkeleyTCPClientDemo.o
 .debug_line    0x000047f0       0x90 Objects - TCPIP Demo App-C32\BerkeleyTCPServerDemo.o
 .debug_line    0x00004880       0x90 ..\Microchip\TCPIP Stack\Objects - TCPIP Demo App-C32\ENCX24J600.o
 .debug_line    0x00004910       0x90 ..\Microchip\TCPIP Stack\Objects - TCPIP Demo App-C32\Random.o
 .debug_line    0x000049a0       0x90 ..\Microchip\TCPIP Stack\Objects - TCPIP Demo App-C32\RSA.o
 .debug_line    0x00004a30       0x90 ..\Microchip\TCPIP Stack\Objects - TCPIP Demo App-C32\SSL.o
 .debug_line    0x00004ac0       0x90 ..\Microchip\TCPIP Stack\Objects - TCPIP Demo App-C32\ARCFOUR.o
 .debug_line    0x00004b50       0x90 ..\Microchip\TCPIP Stack\Objects - TCPIP Demo App-C32\BigInt.o
 .debug_line    0x00004be0       0x90 Objects - TCPIP Demo App-C32\CustomSSLCert.o
 .debug_line    0x00004c70       0xcc Objects - TCPIP Demo App-C32\MPFSImg2-C32.o
 .debug_line    0x00004d3c       0x85 C:/Program Files/Microchip/MPLAB C32/bin/../lib/gcc/pic32mx/3.4.4/../../../../pic32mx/lib/size\libc.a(strchr.o)
 .debug_line    0x00004dc1       0x85 C:/Program Files/Microchip/MPLAB C32/bin/../lib/gcc/pic32mx/3.4.4/../../../../pic32mx/lib/size\libc.a(strstr.o)
 .debug_line    0x00004e46       0x83 C:/Program Files/Microchip/MPLAB C32/bin/../lib/gcc/pic32mx/3.4.4/../../../../pic32mx/lib/size\libc.a(exit.o)
 .debug_line    0x00004ec9       0x83 C:/Program Files/Microchip/MPLAB C32/bin/../lib/gcc/pic32mx/3.4.4/../../../../pic32mx/lib/size\libc.a(rand.o)
 .debug_line    0x00004f4c       0x83 C:/Program Files/Microchip/MPLAB C32/bin/../lib/gcc/pic32mx/3.4.4/../../../../pic32mx/lib/size\libc.a(atol.o)
 .debug_line    0x00004fcf       0x83 C:/Program Files/Microchip/MPLAB C32/bin/../lib/gcc/pic32mx/3.4.4/../../../../pic32mx/lib/size\libc.a(atoi.o)
 .debug_line    0x00005052       0x85 C:/Program Files/Microchip/MPLAB C32/bin/../lib/gcc/pic32mx/3.4.4/../../../../pic32mx/lib/size\libc.a(strtol.o)
 .debug_line    0x000050d7       0x8a C:/Program Files/Microchip/MPLAB C32/bin/../lib/gcc/pic32mx/3.4.4/../../../../pic32mx/lib/size\libc.a(_iobfuncs.o)
 .debug_line    0x00005161       0x86 C:/Program Files/Microchip/MPLAB C32/bin/../lib/gcc/pic32mx/3.4.4/../../../../pic32mx/lib/size\libc.a(stubs.o)
 .debug_line    0x000051e7       0xa4 C:/Program Files/Microchip/MPLAB C32/bin/../lib/gcc/pic32mx/3.4.4/../../../../pic32mx/lib/size\libc.a(default-bootstrap-exception-handler.o)
 .debug_line    0x0000528b       0x91 C:/Program Files/Microchip/MPLAB C32/bin/../lib/gcc/pic32mx/3.4.4/../../../../pic32mx/lib/size\libc.a(default-on-reset.o)
 .debug_line    0x0000531c       0x95 C:/Program Files/Microchip/MPLAB C32/bin/../lib/gcc/pic32mx/3.4.4/../../../../pic32mx/lib/size\libc.a(default-on-bootstrap.o)
 .debug_line    0x000053b1       0x8a C:/Program Files/Microchip/MPLAB C32/bin/../lib/gcc/pic32mx/3.4.4/../../../../pic32mx/lib/size\libc.a(_mon_getc.o)
 .debug_line    0x0000543b       0x8b C:/Program Files/Microchip/MPLAB C32/bin/../lib/gcc/pic32mx/3.4.4/../../../../pic32mx/lib/size\libc.a(_mon_write.o)
 .debug_line    0x000054c6       0x86 C:/Program Files/Microchip/MPLAB C32/bin/../lib/gcc/pic32mx/3.4.4/../../../../pic32mx/lib/size\libc.a(_exit.o)
 .debug_line    0x0000554c       0x8a C:/Program Files/Microchip/MPLAB C32/bin/../lib/gcc/pic32mx/3.4.4/../../../../pic32mx/lib/size\libc.a(_mon_putc.o)
 .debug_line    0x000055d6       0xa9 C:/Program Files/Microchip/MPLAB C32/bin/../lib/gcc/pic32mx/3.4.4/../../../../pic32mx/lib/size\libmchp_peripheral.a(int_disable_interrupts_lib.o)
 .debug_line    0x0000567f       0xa4 C:/Program Files/Microchip/MPLAB C32/bin/../lib/gcc/pic32mx/3.4.4/../../../../pic32mx/lib/size\libmchp_peripheral.a(int_enable_mv_int_lib.o)
 .debug_line    0x00005723       0xa9 C:/Program Files/Microchip/MPLAB C32/bin/../lib/gcc/pic32mx/3.4.4/../../../../pic32mx/lib/size\libmchp_peripheral.a(int_restore_interrupts_lib.o)
 .debug_line    0x000057cc       0x9f C:/Program Files/Microchip/MPLAB C32/bin/../lib/gcc/pic32mx/3.4.4/../../../../pic32mx/lib/size\libmchp_peripheral.a(soft_reset_lib.o)
 .debug_line    0x0000586b       0x98 C:/Program Files/Microchip/MPLAB C32/bin/../lib/gcc/pic32mx/3.4.4/../../../../pic32mx/lib/size\libmchp_peripheral.a(pcache.o)
 .debug_line    0x00005903       0xa8 C:/Program Files/Microchip/MPLAB C32/bin/../lib/gcc/pic32mx/3.4.4/../../../../pic32mx/lib/size\libmchp_peripheral.a(int_enable_interrupts_lib.o)

.debug_frame    0x00000000     0x1ffc
 *(.debug_frame)
 .debug_frame   0x00000000       0xcc Objects - TCPIP Demo App-C32\MainDemo.o
 .debug_frame   0x000000cc       0x90 Objects - TCPIP Demo App-C32\CustomHTTPApp.o
 .debug_frame   0x0000015c       0xc8 ..\Microchip\TCPIP Stack\Objects - TCPIP Demo App-C32\ARP.o
 .debug_frame   0x00000224       0x4c ..\Microchip\TCPIP Stack\Objects - TCPIP Demo App-C32\Delay.o
 .debug_frame   0x00000270       0xc8 ..\Microchip\TCPIP Stack\Objects - TCPIP Demo App-C32\DHCP.o
 .debug_frame   0x00000338       0x70 ..\Microchip\TCPIP Stack\Objects - TCPIP Demo App-C32\DHCPs.o
 .debug_frame   0x000003a8       0xcc ..\Microchip\TCPIP Stack\Objects - TCPIP Demo App-C32\DNS.o
 .debug_frame   0x00000474       0xc4 ..\Microchip\TCPIP Stack\Objects - TCPIP Demo App-C32\DynDNS.o
 .debug_frame   0x00000538      0x3ec ..\Microchip\TCPIP Stack\Objects - TCPIP Demo App-C32\ENC28J60.o
 .debug_frame   0x00000924       0xa8 ..\Microchip\TCPIP Stack\Objects - TCPIP Demo App-C32\Hashes.o
 .debug_frame   0x000009cc      0x1bc ..\Microchip\TCPIP Stack\Objects - TCPIP Demo App-C32\Helpers.o
 .debug_frame   0x00000b88      0x238 ..\Microchip\TCPIP Stack\Objects - TCPIP Demo App-C32\HTTP2.o
 .debug_frame   0x00000dc0       0x30 ..\Microchip\TCPIP Stack\Objects - TCPIP Demo App-C32\ICMP.o
 .debug_frame   0x00000df0       0x90 ..\Microchip\TCPIP Stack\Objects - TCPIP Demo App-C32\IP.o
 .debug_frame   0x00000e80       0x8c ..\Microchip\TCPIP Stack\Objects - TCPIP Demo App-C32\LCDBlocking.o
 .debug_frame   0x00000f0c      0x280 ..\Microchip\TCPIP Stack\Objects - TCPIP Demo App-C32\MPFS2.o
 .debug_frame   0x0000118c       0x70 ..\Microchip\TCPIP Stack\Objects - TCPIP Demo App-C32\NBNS.o
 .debug_frame   0x000011fc      0x19c ..\Microchip\TCPIP Stack\Objects - TCPIP Demo App-C32\SMTP.o
 .debug_frame   0x00001398       0x70 ..\Microchip\TCPIP Stack\Objects - TCPIP Demo App-C32\StackTsk.o
 .debug_frame   0x00001408      0x3a0 ..\Microchip\TCPIP Stack\Objects - TCPIP Demo App-C32\TCP.o
 .debug_frame   0x000017a8       0xe4 ..\Microchip\TCPIP Stack\Objects - TCPIP Demo App-C32\Tick.o
 .debug_frame   0x0000188c      0x228 ..\Microchip\TCPIP Stack\Objects - TCPIP Demo App-C32\UDP.o
 .debug_frame   0x00001ab4       0x30 Objects - TCPIP Demo App-C32\SMTPDemo.o
 .debug_frame   0x00001ae4       0x20 C:/Program Files/Microchip/MPLAB C32/bin/../lib/gcc/pic32mx/3.4.4/../../../../pic32mx/lib/size\libc.a(strchr.o)
 .debug_frame   0x00001b04       0x20 C:/Program Files/Microchip/MPLAB C32/bin/../lib/gcc/pic32mx/3.4.4/../../../../pic32mx/lib/size\libc.a(strstr.o)
 .debug_frame   0x00001b24       0x34 C:/Program Files/Microchip/MPLAB C32/bin/../lib/gcc/pic32mx/3.4.4/../../../../pic32mx/lib/size\libc.a(exit.o)
 .debug_frame   0x00001b58       0x54 C:/Program Files/Microchip/MPLAB C32/bin/../lib/gcc/pic32mx/3.4.4/../../../../pic32mx/lib/size\libc.a(rand.o)
 .debug_frame   0x00001bac       0x28 C:/Program Files/Microchip/MPLAB C32/bin/../lib/gcc/pic32mx/3.4.4/../../../../pic32mx/lib/size\libc.a(atol.o)
 .debug_frame   0x00001bd4       0x28 C:/Program Files/Microchip/MPLAB C32/bin/../lib/gcc/pic32mx/3.4.4/../../../../pic32mx/lib/size\libc.a(atoi.o)
 .debug_frame   0x00001bfc       0x20 C:/Program Files/Microchip/MPLAB C32/bin/../lib/gcc/pic32mx/3.4.4/../../../../pic32mx/lib/size\libc.a(strtol.o)
 .debug_frame   0x00001c1c       0x98 C:/Program Files/Microchip/MPLAB C32/bin/../lib/gcc/pic32mx/3.4.4/../../../../pic32mx/lib/size\libc.a(_iobfuncs.o)
 .debug_frame   0x00001cb4      0x178 C:/Program Files/Microchip/MPLAB C32/bin/../lib/gcc/pic32mx/3.4.4/../../../../pic32mx/lib/size\libc.a(stubs.o)
 .debug_frame   0x00001e2c       0x20 C:/Program Files/Microchip/MPLAB C32/bin/../lib/gcc/pic32mx/3.4.4/../../../../pic32mx/lib/size\libc.a(default-bootstrap-exception-handler.o)
 .debug_frame   0x00001e4c       0x20 C:/Program Files/Microchip/MPLAB C32/bin/../lib/gcc/pic32mx/3.4.4/../../../../pic32mx/lib/size\libc.a(default-on-reset.o)
 .debug_frame   0x00001e6c       0x20 C:/Program Files/Microchip/MPLAB C32/bin/../lib/gcc/pic32mx/3.4.4/../../../../pic32mx/lib/size\libc.a(default-on-bootstrap.o)
 .debug_frame   0x00001e8c       0x20 C:/Program Files/Microchip/MPLAB C32/bin/../lib/gcc/pic32mx/3.4.4/../../../../pic32mx/lib/size\libc.a(_mon_getc.o)
 .debug_frame   0x00001eac       0x30 C:/Program Files/Microchip/MPLAB C32/bin/../lib/gcc/pic32mx/3.4.4/../../../../pic32mx/lib/size\libc.a(_mon_write.o)
 .debug_frame   0x00001edc       0x20 C:/Program Files/Microchip/MPLAB C32/bin/../lib/gcc/pic32mx/3.4.4/../../../../pic32mx/lib/size\libc.a(_exit.o)
 .debug_frame   0x00001efc       0x20 C:/Program Files/Microchip/MPLAB C32/bin/../lib/gcc/pic32mx/3.4.4/../../../../pic32mx/lib/size\libc.a(_mon_putc.o)
 .debug_frame   0x00001f1c       0x20 C:/Program Files/Microchip/MPLAB C32/bin/../lib/gcc/pic32mx/3.4.4/../../../../pic32mx/lib/size\libmchp_peripheral.a(int_disable_interrupts_lib.o)
 .debug_frame   0x00001f3c       0x28 C:/Program Files/Microchip/MPLAB C32/bin/../lib/gcc/pic32mx/3.4.4/../../../../pic32mx/lib/size\libmchp_peripheral.a(int_enable_mv_int_lib.o)
 .debug_frame   0x00001f64       0x20 C:/Program Files/Microchip/MPLAB C32/bin/../lib/gcc/pic32mx/3.4.4/../../../../pic32mx/lib/size\libmchp_peripheral.a(int_restore_interrupts_lib.o)
 .debug_frame   0x00001f84       0x28 C:/Program Files/Microchip/MPLAB C32/bin/../lib/gcc/pic32mx/3.4.4/../../../../pic32mx/lib/size\libmchp_peripheral.a(soft_reset_lib.o)
 .debug_frame   0x00001fac       0x30 C:/Program Files/Microchip/MPLAB C32/bin/../lib/gcc/pic32mx/3.4.4/../../../../pic32mx/lib/size\libmchp_peripheral.a(pcache.o)
 .debug_frame   0x00001fdc       0x20 C:/Program Files/Microchip/MPLAB C32/bin/../lib/gcc/pic32mx/3.4.4/../../../../pic32mx/lib/size\libmchp_peripheral.a(int_enable_interrupts_lib.o)

.debug_str      0x00000000     0x14a2
 *(.debug_str)
 .debug_str     0x00000000       0x40 Objects - TCPIP Demo App-C32\MainDemo.o
 .debug_str     0x00000040       0x1b Objects - TCPIP Demo App-C32\CustomHTTPApp.o
 .debug_str     0x0000005b       0x12 ..\Microchip\TCPIP Stack\Objects - TCPIP Demo App-C32\UDPPerformanceTest.o
 .debug_str     0x0000006d       0x12 ..\Microchip\TCPIP Stack\Objects - TCPIP Demo App-C32\Announce.o
 .debug_str     0x0000007f       0x20 ..\Microchip\TCPIP Stack\Objects - TCPIP Demo App-C32\ARP.o
 .debug_str     0x0000009f       0x12 ..\Microchip\TCPIP Stack\Objects - TCPIP Demo App-C32\Delay.o
 .debug_str     0x000000b1       0x12 ..\Microchip\TCPIP Stack\Objects - TCPIP Demo App-C32\DHCP.o
 .debug_str     0x000000c3       0x12 ..\Microchip\TCPIP Stack\Objects - TCPIP Demo App-C32\DHCPs.o
 .debug_str     0x000000d5       0x12 ..\Microchip\TCPIP Stack\Objects - TCPIP Demo App-C32\DNS.o
 .debug_str     0x000000e7       0x4b ..\Microchip\TCPIP Stack\Objects - TCPIP Demo App-C32\DynDNS.o
 .debug_str     0x00000132       0x7f ..\Microchip\TCPIP Stack\Objects - TCPIP Demo App-C32\ENC28J60.o
 .debug_str     0x000001b1       0x12 ..\Microchip\TCPIP Stack\Objects - TCPIP Demo App-C32\FTP.o
 .debug_str     0x000001c3       0x19 ..\Microchip\TCPIP Stack\Objects - TCPIP Demo App-C32\Hashes.o
 .debug_str     0x000001dc       0x3c ..\Microchip\TCPIP Stack\Objects - TCPIP Demo App-C32\Helpers.o
 .debug_str     0x00000218       0x2a ..\Microchip\TCPIP Stack\Objects - TCPIP Demo App-C32\HTTP2.o
 .debug_str     0x00000242       0x12 ..\Microchip\TCPIP Stack\Objects - TCPIP Demo App-C32\HTTP.o
 .debug_str     0x00000254       0x12 ..\Microchip\TCPIP Stack\Objects - TCPIP Demo App-C32\ICMP.o
 .debug_str     0x00000266       0x1b ..\Microchip\TCPIP Stack\Objects - TCPIP Demo App-C32\IP.o
 .debug_str     0x00000281       0x12 ..\Microchip\TCPIP Stack\Objects - TCPIP Demo App-C32\LCDBlocking.o
 .debug_str     0x00000293       0x2b ..\Microchip\TCPIP Stack\Objects - TCPIP Demo App-C32\MPFS2.o
 .debug_str     0x000002be       0x12 ..\Microchip\TCPIP Stack\Objects - TCPIP Demo App-C32\MPFS.o
 .debug_str     0x000002d0       0x1d ..\Microchip\TCPIP Stack\Objects - TCPIP Demo App-C32\NBNS.o
 .debug_str     0x000002ed       0x12 ..\Microchip\TCPIP Stack\Objects - TCPIP Demo App-C32\Reboot.o
 .debug_str     0x000002ff       0x5a ..\Microchip\TCPIP Stack\Objects - TCPIP Demo App-C32\SMTP.o
 .debug_str     0x00000359       0x12 ..\Microchip\TCPIP Stack\Objects - TCPIP Demo App-C32\SNMP.o
 .debug_str     0x0000036b       0x12 ..\Microchip\TCPIP Stack\Objects - TCPIP Demo App-C32\SNTP.o
 .debug_str     0x0000037d       0x12 ..\Microchip\TCPIP Stack\Objects - TCPIP Demo App-C32\SPIEEPROM.o
 .debug_str     0x0000038f       0x12 ..\Microchip\TCPIP Stack\Objects - TCPIP Demo App-C32\SPIFlash.o
 .debug_str     0x000003a1       0x12 ..\Microchip\TCPIP Stack\Objects - TCPIP Demo App-C32\SPIRAM.o
 .debug_str     0x000003b3       0x12 ..\Microchip\TCPIP Stack\Objects - TCPIP Demo App-C32\StackTsk.o
 .debug_str     0x000003c5       0xa7 ..\Microchip\TCPIP Stack\Objects - TCPIP Demo App-C32\TCP.o
 .debug_str     0x0000046c       0x12 ..\Microchip\TCPIP Stack\Objects - TCPIP Demo App-C32\TCPPerformanceTest.o
 .debug_str     0x0000047e       0x12 ..\Microchip\TCPIP Stack\Objects - TCPIP Demo App-C32\Telnet.o
 .debug_str     0x00000490       0x12 ..\Microchip\TCPIP Stack\Objects - TCPIP Demo App-C32\TFTPc.o
 .debug_str     0x000004a2       0x12 ..\Microchip\TCPIP Stack\Objects - TCPIP Demo App-C32\Tick.o
 .debug_str     0x000004b4       0x12 ..\Microchip\TCPIP Stack\Objects - TCPIP Demo App-C32\UART2TCPBridge.o
 .debug_str     0x000004c6       0x12 ..\Microchip\TCPIP Stack\Objects - TCPIP Demo App-C32\UART.o
 .debug_str     0x000004d8       0x48 ..\Microchip\TCPIP Stack\Objects - TCPIP Demo App-C32\UDP.o
 .debug_str     0x00000520       0x12 Objects - TCPIP Demo App-C32\CustomSNMPApp.o
 .debug_str     0x00000532       0x12 Objects - TCPIP Demo App-C32\UARTConfig.o
 .debug_str     0x00000544       0x12 Objects - TCPIP Demo App-C32\GenericTCPClient.o
 .debug_str     0x00000556       0x12 Objects - TCPIP Demo App-C32\GenericTCPServer.o
 .debug_str     0x00000568       0x12 Objects - TCPIP Demo App-C32\LegacyHTTPApp.o
 .debug_str     0x0000057a       0x12 Objects - TCPIP Demo App-C32\PingDemo.o
 .debug_str     0x0000058c       0x3d Objects - TCPIP Demo App-C32\SMTPDemo.o
 .debug_str     0x000005c9       0x12 ..\Microchip\TCPIP Stack\Objects - TCPIP Demo App-C32\BerkeleyAPI.o
 .debug_str     0x000005db       0x12 Objects - TCPIP Demo App-C32\BerkeleyUDPClientDemo.o
 .debug_str     0x000005ed       0x12 Objects - TCPIP Demo App-C32\BerkeleyTCPClientDemo.o
 .debug_str     0x000005ff       0x12 Objects - TCPIP Demo App-C32\BerkeleyTCPServerDemo.o
 .debug_str     0x00000611       0x12 ..\Microchip\TCPIP Stack\Objects - TCPIP Demo App-C32\ENCX24J600.o
 .debug_str     0x00000623       0x12 ..\Microchip\TCPIP Stack\Objects - TCPIP Demo App-C32\Random.o
 .debug_str     0x00000635       0x12 ..\Microchip\TCPIP Stack\Objects - TCPIP Demo App-C32\RSA.o
 .debug_str     0x00000647       0x12 ..\Microchip\TCPIP Stack\Objects - TCPIP Demo App-C32\SSL.o
 .debug_str     0x00000659       0x12 ..\Microchip\TCPIP Stack\Objects - TCPIP Demo App-C32\ARCFOUR.o
 .debug_str     0x0000066b       0x12 ..\Microchip\TCPIP Stack\Objects - TCPIP Demo App-C32\BigInt.o
 .debug_str     0x0000067d       0x12 Objects - TCPIP Demo App-C32\CustomSSLCert.o
 .debug_str     0x0000068f       0x12 Objects - TCPIP Demo App-C32\MPFSImg2-C32.o
 .debug_str     0x000006a1       0xb6 C:/Program Files/Microchip/MPLAB C32/bin/../lib/gcc/pic32mx/3.4.4/../../../../pic32mx/lib/size\libc.a(strchr.o)
 .debug_str     0x00000757       0x6f C:/Program Files/Microchip/MPLAB C32/bin/../lib/gcc/pic32mx/3.4.4/../../../../pic32mx/lib/size\libc.a(strstr.o)
                                 0xb6 (size before relaxing)
 .debug_str     0x000007c6       0x66 C:/Program Files/Microchip/MPLAB C32/bin/../lib/gcc/pic32mx/3.4.4/../../../../pic32mx/lib/size\libc.a(exit.o)
                                 0xb2 (size before relaxing)
 .debug_str     0x0000082c       0x73 C:/Program Files/Microchip/MPLAB C32/bin/../lib/gcc/pic32mx/3.4.4/../../../../pic32mx/lib/size\libc.a(rand.o)
                                 0xbf (size before relaxing)
 .debug_str     0x0000089f       0x6b C:/Program Files/Microchip/MPLAB C32/bin/../lib/gcc/pic32mx/3.4.4/../../../../pic32mx/lib/size\libc.a(atol.o)
                                 0xb2 (size before relaxing)
 .debug_str     0x0000090a       0x6b C:/Program Files/Microchip/MPLAB C32/bin/../lib/gcc/pic32mx/3.4.4/../../../../pic32mx/lib/size\libc.a(atoi.o)
                                 0xb2 (size before relaxing)
 .debug_str     0x00000975       0x6f C:/Program Files/Microchip/MPLAB C32/bin/../lib/gcc/pic32mx/3.4.4/../../../../pic32mx/lib/size\libc.a(strtol.o)
                                 0xb6 (size before relaxing)
 .debug_str     0x000009e4       0xb7 C:/Program Files/Microchip/MPLAB C32/bin/../lib/gcc/pic32mx/3.4.4/../../../../pic32mx/lib/size\libc.a(_iobfuncs.o)
                                 0xfe (size before relaxing)
 .debug_str     0x00000a9b      0x2d9 C:/Program Files/Microchip/MPLAB C32/bin/../lib/gcc/pic32mx/3.4.4/../../../../pic32mx/lib/size\libc.a(stubs.o)
                                0x320 (size before relaxing)
 .debug_str     0x00000d74       0xa4 C:/Program Files/Microchip/MPLAB C32/bin/../lib/gcc/pic32mx/3.4.4/../../../../pic32mx/lib/size\libc.a(default-bootstrap-exception-handler.o)
                                 0xeb (size before relaxing)
 .debug_str     0x00000e18       0x7e C:/Program Files/Microchip/MPLAB C32/bin/../lib/gcc/pic32mx/3.4.4/../../../../pic32mx/lib/size\libc.a(default-on-reset.o)
                                 0xc5 (size before relaxing)
 .debug_str     0x00000e96       0x86 C:/Program Files/Microchip/MPLAB C32/bin/../lib/gcc/pic32mx/3.4.4/../../../../pic32mx/lib/size\libc.a(default-on-bootstrap.o)
                                 0xcd (size before relaxing)
 .debug_str     0x00000f1c       0x77 C:/Program Files/Microchip/MPLAB C32/bin/../lib/gcc/pic32mx/3.4.4/../../../../pic32mx/lib/size\libc.a(_mon_getc.o)
                                 0xbe (size before relaxing)
 .debug_str     0x00000f93       0x79 C:/Program Files/Microchip/MPLAB C32/bin/../lib/gcc/pic32mx/3.4.4/../../../../pic32mx/lib/size\libc.a(_mon_write.o)
                                 0xc0 (size before relaxing)
 .debug_str     0x0000100c       0x6f C:/Program Files/Microchip/MPLAB C32/bin/../lib/gcc/pic32mx/3.4.4/../../../../pic32mx/lib/size\libc.a(_exit.o)
                                 0xb6 (size before relaxing)
 .debug_str     0x0000107b       0x77 C:/Program Files/Microchip/MPLAB C32/bin/../lib/gcc/pic32mx/3.4.4/../../../../pic32mx/lib/size\libc.a(_mon_putc.o)
                                 0xbe (size before relaxing)
 .debug_str     0x000010f2       0xa1 C:/Program Files/Microchip/MPLAB C32/bin/../lib/gcc/pic32mx/3.4.4/../../../../pic32mx/lib/size\libmchp_peripheral.a(int_disable_interrupts_lib.o)
                                 0xe8 (size before relaxing)
 .debug_str     0x00001193       0xa7 C:/Program Files/Microchip/MPLAB C32/bin/../lib/gcc/pic32mx/3.4.4/../../../../pic32mx/lib/size\libmchp_peripheral.a(int_enable_mv_int_lib.o)
                                 0xee (size before relaxing)
 .debug_str     0x0000123a       0xa1 C:/Program Files/Microchip/MPLAB C32/bin/../lib/gcc/pic32mx/3.4.4/../../../../pic32mx/lib/size\libmchp_peripheral.a(int_restore_interrupts_lib.o)
                                 0xe8 (size before relaxing)
 .debug_str     0x000012db       0x8c C:/Program Files/Microchip/MPLAB C32/bin/../lib/gcc/pic32mx/3.4.4/../../../../pic32mx/lib/size\libmchp_peripheral.a(soft_reset_lib.o)
                                 0xd3 (size before relaxing)
 .debug_str     0x00001367       0x9c C:/Program Files/Microchip/MPLAB C32/bin/../lib/gcc/pic32mx/3.4.4/../../../../pic32mx/lib/size\libmchp_peripheral.a(pcache.o)
                                 0xe3 (size before relaxing)
 .debug_str     0x00001403       0x9f C:/Program Files/Microchip/MPLAB C32/bin/../lib/gcc/pic32mx/3.4.4/../../../../pic32mx/lib/size\libmchp_peripheral.a(int_enable_interrupts_lib.o)
                                 0xe6 (size before relaxing)

.debug_loc
 *(.debug_loc)

.debug_macinfo
 *(.debug_macinfo)

.debug_weaknames
 *(.debug_weaknames)

.debug_funcnames
 *(.debug_funcnames)

.debug_typenames
 *(.debug_typenames)

.debug_varnames
 *(.debug_varnames)

/DISCARD/
 *(.note.GNU-stack)
OUTPUT(TCPIP Demo App-C32.elf elf32-tradlittlemips)

.mdebug.abi32   0x9d01db80        0x0

.rel.dyn        0x9d01db80        0x0
